:100000000C94C0030C94DD030C94DD030C94DD030D
:100010000C94DD030C94DD030C94DD030C94DD03E0
:100020000C94DD030C94380E0C94DD030C94DD036A
:100030000C94CE190C94DD030C94DD030C949A19E6
:100040000C94DD030C94DD030C94630D0C94DD0320
:100050000C9479090C94DD030C949A050C94DD033F
:100060000C940D0F0C94DD030C94D1180C94DD034B
:100070000C94B63E0C94DD030C94DD030A0A0D00CB
:100080004E65757472616C0048656164696E67489D
:100090006F6C64000A0D436F6E74726F6C3A2000CF
:1000A0000A0D537570706F727420666F722047501E
:1000B0005320617420326E642055415254000A0D61
:1000C000537570706F727420666F722047505320A2
:1000D0006174203173742055415254000A0D5375D8
:1000E00070706F727420666F72204D4B334D4147B4
:1000F00020436F6D70617373004F4B0A0D000A0D42
:1001000043616C6962726174696E67206169722013
:1001100070726573737572652073656E736F722E7E
:100120002E000A0D414343206E6F742063616C6999
:1001300062726174656421000A0D3D3D3D3D3D3DA7
:100140003D3D3D3D3D3D3D3D3D3D3D3D3D3D3D3DDF
:100150003D3D3D3D3D3D3D3D000A0D466C696768B6
:1001600074436F6E74726F6C0A0D486172647761CC
:1001700072653A25642E25640A0D536F66747761A3
:1001800072653A5625642E2564256320002E0041B1
:100190006C743A2025642E252E3364206D004C614A
:1001A000743A2025642E252E3364252E3364206472
:1001B0006567004C6F6E3A2025642E252E3364252A
:1001C0002E33642064656700536174733A2025649C
:1001D000204669783A203F3F00536174733A2025E6
:1001E00064204669783A20334400536174733A209E
:1001F0002564204669783A20324400536174733A8A
:10020000202564204669783A204E6F004E6F2047C3
:1002100050532064617461210048693A2534692093
:100220002043663A253469200047733A2534692013
:100230002059613A25346920004E693A25346920F5
:1002400020526F3A253469200045787465726E43F8
:100250006F6E74726F6C20200052616E67653A2574
:1002600033692D25336900506F736974696F6E3A75
:100270002025336900536574706F696E74202025E2
:10028000336900536572766F202000506F343A2036
:1002900025336920506F383A2025336900506F3379
:1002A0003A2025336920506F373A202533690050B2
:1002B0006F323A2025336920506F363A2025336952
:1002C00000506F313A2025336920506F353A202590
:1002D0003369004F6666436F757273653A20253542
:1002E000690048656164696E673A20202025356998
:1002F00000436F757273653A202020202535690010
:10030000436F6D70617373202020202020200052E5
:10031000432D4C6576656C3A2025356900566F6C27
:10032000746167653A20202535690048656967680A
:10033000742025346920282533692900526F6C6C9C
:10034000202020253469202825336929004E69633F
:100350006B20202534692028253369290041434337
:10036000202D2053656E736F720059617720202015
:1003700025346920282533692900526F6C6C2020B0
:10038000253469202825336929004E69636B2025AF
:1003900034692028253369290059617720202025D8
:1003A000346920282533692900526F6C6C20202580
:1003B0003469202825336929004E69636B20253470
:1003C00069202825336929004779726F202D205331
:1003D000656E736F720050333A25346920205034B3
:1003E0003A253469200050313A25346920205032B2
:1003F0003A253469200047733A2534692020596131
:100400003A25346920004E693A2534692020526F1C
:100410003A253469200043373A253469202043388F
:100420003A253469200043353A2534692020433683
:100430003A253469200043333A2534692020433477
:100440003A253469200043313A253469202043326B
:100450003A253469200048656164696E673A202056
:100460002025356900526F6C6C3A20202020202016
:10047000253569004E69636B3A2020202020253500
:1004800069004174746974756465004865696768DA
:100490007420436F6E74726F6C004E6F20004F6655
:1004A00066736574202020203A2535690041697201
:1004B0002050726573732E3A253569005365742098
:1004C000506F696E743A2025356900486569676820
:1004D000743A202020202535690028632920486FA0
:1004E0006C67657220427573730053657474696E2E
:1004F000673A202564200048573A5625642E256423
:100500002053573A25642E25642563002B204D691E
:100510006B726F4B6F70746572202B005B25695D89
:10052000005B25695D000A0D5573696E6720506197
:1005300072616D6574657220536574202564000ACC
:100540000D496E69742E20454550524F4D3A204753
:10055000656E65726174696E672044656661756C6D
:10056000742D506172616D657465722E2E2E0000BF
:10057000008F001E01AD013B02CA025803E603745E
:100580000402058F051B06A7063307BE074808D2DD
:10059000085B09E3096B0AF20A780BFD0B810C0476
:1005A0000D860D070E870E060F840F00107B10F5C9
:1005B000106E11E5115B12CF124213B31323149284
:1005C00014FE146A15D3153B16A11605176717C834
:1005D0001727188318DE1837198E19E319361A876A
:1005E0001AD61A231B6E1BB61BFD1B411C831CC392
:1005F0001C001D3C1D751DAB1DE01D121E421E6F13
:100600001E9A1EC31EE91E0D1F2E1F4D1F691F843B
:100610001F9B1FB01FC31FD31FE11FEC1FF51FFB44
:100620001FFF1F002000010203040405060708093C
:100630000A0B0B0C0D0E0F101111121314151516B9
:10064000171818191A1B1B1C1D1D1E1F1F202121E6
:1006500022232324242525262727282829292A2A36
:100660002B2B2C2C2D2D2D2E2E2F2F3030303131A9
:100670003232323333333434343535353636363737
:10068000373737383838393939393A3A3A3A3B3BDB
:100690003B3B3C3C3C3C3C3D3D3D3D3E3E3E3E3E8E
:1006A0003F3F3F3F3F3F404040404040414141414C
:1006B0004141424242424242424343434343434315
:1006C00044444444444444444545454545454545E2
:1006D00045464646464646464646474747474747B5
:1006E000474747474748484848484848484848488F
:1006F00049494949494949494949494949494A4A68
:100700004A4A4A4A4A4A4A4A4A4A4A4A4B4B4B4B45
:100710004B4B4B4B4B4B4B4B4B4B4B4B4B4C4C4C26
:100720004C4C4C4C4C4C4C4C4C4C4C4C4C4C4C4C09
:100730004D4D4D4D4D4D4D4D4D4D4D4D4D4D4D4DE9
:100740004D4D4D4D4D4D4E4E4E4E4E4E4E4E4E4ECF
:100750004E4E4E4E4E4E4E4E4E4E4E4E4E4E4E4EB9
:100760004F4F4F4F4F4F4F4F4F4F4F4F4F4F4F4F99
:100770004F4F4F4F4F4F4F4F4F4F4F4F4F4F4F00D8
:1007800011241FBECFEFD0E1DEBFCDBF14E0A0E04B
:10079000B1E0ECE1F7E902C005900D92A83BB1078A
:1007A000D9F719E0A8EBB4E001C01D92AA39B1074E
:1007B000E1F70E94DF030C948D4B0C940000CF9363
:1007C000DF93F89414B815B8189B02C08BE001C0F1
:1007D0008AE08093000184B1836084B92091000194
:1007E0002A3011F4289A01C02898299884B7877F65
:1007F00084BF8091600088618093600010926000E7
:1008000080ED97E09093D4048093D30410924B082A
:1008100010924A0810927305109272051092710599
:100820001092700510926F0510926E052A3011F427
:10083000289801C0289A0E9421180E94190D0E9430
:10084000150E0E94D106809100018B3011F40E9498
:10085000593E0E9466190E94F00E0E947A180E946A
:10086000E13E78941092480785E48093490787E039
:1008700080934A0720910001822F6AE00E94BE4ABD
:10088000492F50E0822F0E94BE4A90E02BE630E0D4
:100890003F932F9325E430E03F932F931F921F92B5
:1008A0005F934F939F938F9389E591E09F938F93ED
:1008B0001F920E94750A88E391E09F938F931F9285
:1008C0000E94750A299A0E94A23D84E00E94A23BE0
:1008D0002DB73EB7205F3F4F0FB6F8943EBF0FBE17
:1008E0002DBF8050944050F082E291E09F938F930F
:1008F0001F920E94750A0F900F900F9084EF91E065
:100900000E944E0DEC01CE010E94570D8823D9F3B1
:100910008091B60880FF20C08EEF90E09F938F9368
:100920001F920E94750A88EE93E00E944E0DEC0122
:100930000E94EC110F900F900F90CE010E94570D66
:100940008823D9F389EF90E09F938F931F920E94A1
:10095000750A0F900F900F908CED90E09F938F93FE
:100960001F920E94750A0F900F900F9080910001C6
:100970008A3019F48EEB90E002C080EA90E09F93F9
:100980008F931F920E94750A0F900F900F900E94F4
:10099000B623809100018A3011F4289801C0289A6A
:1009A00080ED97E09093D4048093D30485E5809301
:1009B000520784E990E09F938F931F920E94750ADB
:1009C0008091B6080F900F900F9082FF03C088E8C7
:1009D00090E002C080E890E09F938F931F920E9466
:1009E000750A0F900F900F908CE790E09F938F9374
:1009F0001F920E94750A0E942C1280ED97E090933E
:100A00006D0380936C030F900F900F908091D00432
:100A10008823E1F31092D0040E9460250E947F2376
:100A2000209100012A3011F4289801C0289A809161
:100A30000301882321F081508093030112C010929A
:100A4000C4041092C50410925C0710927F051092A6
:100A50007E051092810510928005109283051092F8
:100A6000820580916C0390916D03892B01F585E0DF
:100A700090E090936D0380936C030E94A118809185
:100A80000403909105038F5F9F4FF9F480915A05FD
:100A90008823D9F080E197E29093D4048093D30423
:100AA00080E890E090930503809304030EC080914A
:100AB0006C0390916D03019790936D0380936C0389
:100AC0002A3011F4289801C0289A8091D0048823F4
:100AD00021F080915A05882311F40E9440070E945A
:100AE0003C08CE010E94570D882309F48FCF209136
:100AF0000803309109038091C60890E02817390750
:100B00009CF480910403909105038F5F9F4F61F4E3
:100B100080E797E19093D4048093D30480E093E03E
:100B2000909305038093040384E190E00E944E0DAE
:100B3000EC016CCF1F920F920FB60F9211248F937E
:100B40009F93EF93FF93809102018823E1F48091BA
:100B5000CC049091CD0401969093CD048093CC0465
:100B6000FC01E156F84FE081ED3019F0863991052E
:100B700039F41092CD041092CC0481E080930201EC
:100B8000E093C60004C01092CD041092CC04FF91F3
:100B9000EF919F918F910F900FBE0F901F9018951E
:100BA000DC0120E030E040E050E008C0FA01E1560E
:100BB000F84F8081280F311D4F5F5F4F4A175B0749
:100BC000A9F73F70C90136E0969587953A95E1F708
:100BD000835CFD01E156F84F808311962F73235CEF
:100BE000FD01E156F84F2083A056B84F8DE08C935D
:100BF0001092020180919F078093C60008951F9371
:100C0000CF93DF93EA01722F93E290939F07609353
:100C1000A0078093A107A3E0B0E060E04FC0FE0111
:100C2000E60FF11D90816F5F715019F410E040E004
:100C30000FC0FE01E60FF11D40816F5F715011F48E
:100C400010E006C0FE01E60FF11D10816F5F7150CC
:100C5000892F86958695835CFD01E156F84F808348
:100C600050E09A0184E0369527958A95E1F7892F1F
:100C700090E083709070F4E0880F991FFA95E1F787
:100C8000282B235CFD01E056F84F2083812F8295AD
:100C90008695869583704F705070440F551F440F92
:100CA000551F842B835CFD01EF55F84F80831F7324
:100CB000135CFD01EE55F84F10831496772309F06D
:100CC000AECFCD010E94D005DF91CF911F91089545
:100CD0001F93CF93DF93EC0170E0A22FB0E0129747
:100CE00048C0E42FF0E0E255F94F30814F5FE42F28
:100CF000F0E0E255F94F50814F5FE42FF0E0E2550C
:100D0000F94F10814F5FE42FF0E0E255F94F208159
:100D10004F5F842F90E0A817B90774F15D53FE016F
:100D2000E70FF11D852F82958F703D53330F330FE1
:100D3000382B3083613001F1912F9D537F5FFE018D
:100D4000E70FF11D71505295507F892F869586953A
:100D5000582B508363506F3F79F07E5FFE01E70FA1
:100D6000F11D9295990F990F907C2D53922B9083A2
:100D70007F5F662309F0B5CFDF91CF911F91089572
:100D80001F93182F8A3019F48DE00E94C0068091BD
:100D9000C00085FFFCCF1093C60080E090E01F915B
:100DA00008951F931FB7F8948091C1008F778093A7
:100DB000C1008091C1008F7B8093C100589A5098E8
:100DC000599A519A1092C5008AE28093C40080918A
:100DD000C00082608093C00088E18093C100809150
:100DE000C2008F778093C2008091C2008F7B809376
:100DF000C2008091C2008F7D8093C2008091C200AA
:100E00008F7E8093C2008091C200877F8093C20052
:100E10008091C1008B7F8093C1008091C20084606B
:100E20008093C2008091C20082608093C20002C0A1
:100E30008091C6008091C00087FDFACF8091C100EB
:100E400080688093C1008091C10080648093C1005C
:100E50001092BE0481E08093020188EC90E00E9431
:100E60004E0D90934707809346078CED90E00E94CB
:100E70004E0D90934507809344071FBF1F9108951F
:100E800080910201882309F4F6C08091B904882377
:100E900071F080910201882351F06091C8042BE029
:100EA00042E557E087E40E94FF051092B904809163
:100EB0004407909145070E94570D882309F44BC0C1
:100EC00080910201882309F446C060911C0570914D
:100ED0001D0580911E0590911F052CE630E040E035
:100EE00050E00E94134B3093930920939209609134
:100EF00024057091250580912605909127052CE603
:100F000030E040E050E00E94134B3093950920936D
:100F1000940980918B038093960980918C03809330
:100F2000970980915205809398096091C80428E040
:100F300042E959E087E70E94FF058091520585301C
:100F400010F01092520583E690E00E944E0D9093AF
:100F500045078093440780914607909147070E9478
:100F6000570D882321F48091BB048823B1F0809130
:100F70000201882391F06091C80422E44DE557E016
:100F800084E40E94FF051092BB048AEF90E00E9467
:100F90004E0D9093470780934607609101016F3F84
:100FA00089F0462F50E094E0440F551F9A95E1F7E1
:100FB0004C5F5E4F605D20E181E40E94FF058FEF92
:100FC00080930101909135089923A1F0809102014D
:100FD000882381F083E280939F079093A0078DE0A0
:100FE0008093A107109202011092350880919F070B
:100FF0008093C6008091BA04882359F18091020140
:10100000882339F10E9435121092BA043091BD0440
:10101000932F9F5F9093BD04943021F08091BC0486
:10102000882359F02EE146E458E060E084E30E9412
:10103000FF058FEF8093BD040CC044E1949FA00195
:101040001124465E5C4F24E160E0832F8F5C0E9498
:10105000FF058091B804882371F0809102018823F4
:1010600051F06091C8042AE048E457E086E50E9408
:10107000FF051092B80408951F93CF93DF93CDB767
:10108000DEB724970FB6F894DEBF0FBECDBF8091B8
:10109000BE04882309F423C18091B006883609F480
:1010A00086C0893690F4823609F453C0833630F412
:1010B0008B34F1F0813609F010C13FC0833609F45A
:1010C0005CC0873609F009C1A7C0813738F48C3677
:1010D00008F0D0C08B3609F000C18DC0843709F408
:1010E00081C0863709F494C0813709F0F6C098C0F2
:1010F0002091BF0443E062E0CE0101960E946806A1
:1011000089819A8190936F0380936E0380916E031F
:1011100090916F032091700330917103845E9D4F15
:10112000821B930B68E671E00E94DE4A845B90406C
:101130009093510580935005D0C02091BF0443E0A7
:1011400062E0CE0103960E9468068B8180930101C4
:101150002AC02091BF0443E06BE082E597E00E9443
:1011600068068091F60490915407892B8093F604C9
:1011700080915B0780933508B0C02091BF0443E0A5
:101180006BE082E597E00E9468068091F6049091FA
:101190005407892B8093F60480915B078093350870
:1011A00081E08093BB048FEF8093030196C0209170
:1011B000BF0443E062E0CE0103960E94680680917E
:1011C000F6049B81892B8093F6048C818F3F21F458
:1011D00081E08093BC0402C01092BC0481E0809343
:1011E000BA047BC02091BF0443E064E080EC94E04B
:1011F0000E946806D8CF2091BF0443E064E084ECED
:1012000094E00E9468068091C70480933508CBCF94
:1012100081E08093B80461C081E08093B9045DC02F
:101220002091BF0443E062E0CE0103960E9468066D
:10123000809102018823E1F38B818F3F71F086302A
:1012400010F085E08B838B810E94D03B6091C804B5
:101250008B8126E44EEA58E009C01091C80482E070
:101260000E94913B26E44EEA58E0612F855B0E9484
:10127000FF0533C02091BF0443E066E48EEA98E0A6
:101280000E9468068091B0068B560E94BB3B60911D
:10129000D90870E080E090E024EC39E040E050E0D4
:1012A0000E949F4A60937403709375038093760342
:1012B000909377036091DA0870E080E090E00E94FC
:1012C0009F4A609378037093790380937A03909395
:1012D0007B030E94933D0E941B251092BE0424961E
:1012E0000FB6F894DEBF0FBECDBFDF91CF911F9137
:1012F00008951F920F920FB60F9211241F932F93F0
:101300003F934F935F936F937F938F939F93AF938D
:10131000BF93CF93DF93EF93FF931091C60080911B
:1013200000018A3019F4812F0E94EB458091BE04A0
:10133000882309F06DC06091C904662371F41332EB
:1013400079F41093AE0681E08093C90483E290E0C3
:101350009093CB048093CA045BC0663908F054C0F4
:10136000A62FB0E02091CA043091CB041D3069F063
:10137000A255B94F1C936F5F6093C904210F311DB3
:101380003093CB042093CA0443C0FD01E455F94FC8
:101390009081ED01C355D94F8881A901491B51099D
:1013A000481B51095F705093CB044093CA042081BD
:1013B000CA0136E0969587953A95E1F7835C8217E6
:1013C000F1F49881842F8F73835C8917C1F481E0D5
:1013D0008093BE046093BF04A255B94F1C938091C3
:1013E000B006823571F488E190E02CE00FB6F894F5
:1013F000A895809360000FBE2093600002C01092F9
:10140000BE041092C90404C01092C9041092BE0414
:10141000FF91EF91DF91CF91BF91AF919F918F910C
:101420007F916F915F914F913F912F911F910F90FD
:101430000FBE0F901F901895982F8091360881301D
:1014400069F48091F504E82FF0E0E65EFC4F9083AC
:101450008F5F8093F50421E030E005C0892F0E9462
:10146000C006282F30E0C90108951F93182F04C02B
:1014700080E30E941C0A11501116D4F31F910895A5
:101480001F93182F04C080E20E941C0A11501116ED
:10149000D4F31F9108950F931F93CF93DF938C0183
:1014A000EB0108C0F8010F5F1F4FE4918E2F0E94DF
:1014B0001C0A21972097B1F7DF91CF911F910F91CF
:1014C00008950F931F93CF93DF938C01EB0106C018
:1014D000F80181918F010E941C0A21972097C1F782
:1014E000DF91CF911F910F9108952F923F924F92CC
:1014F0005F926F927F928F929F92AF92BF92CF92A4
:10150000DF92EF92FF920F931F93CF93DF93CDB7AC
:10151000DEB7E5970FB6F894DEBF0FBECDBF2B96B2
:101520008FAD2B9780933608CE01835B9F4F9B83B3
:101530008A832D964EAC5FAC2D971EA61FA618AAC7
:1015400019AA9E01225D3F4F3DAB2CAB820102C028
:101550000F5F1F4FF801F490FF2019F0F5E2FF161E
:10156000B9F7B8016419750919F0C2010E944B0A54
:10157000FF2009F445C228010894411C511C19821E
:10158000AA81BB8133241BAA2FEF2AABF201089456
:10159000411C511CB490632D70E06170707035E790
:1015A000B31621F08B2D80628837C9F4611571055F
:1015B00059F02D913D914D915C9113972EA73FA726
:1015C00048AB59AB14960BC08D919C9111979C011F
:1015D00040E050E02EA73FA748AB59AB129630E24F
:1015E000B31621F48981882389F61CC043E2B4161E
:1015F00011F458E055C08AE2B81621F09DE2B91600
:1016000071F408C0FD011296E081EBABE7FFBECF9D
:10161000E195EBABE0E13E2AFFED3F22B7CF2BE2B5
:10162000B21611F4B982B2CF3EE2B31699F5F201C7
:101630000894411C511C84918A3221F0B82E20E07C
:1016400030E01DC0FD0112964081518157FF02C05C
:101650004FEF5FEF4AAB9ACFC90153E0880F991F54
:101660005A95E1F7220F331F280F391F2B0D311D1B
:1016700020533040F2010894411C511CB4908B2D32
:1016800080538A3048F3A90137FF02C04FEF5FEF64
:101690004AAB85CF40E3B41629F434FC77CF50E24F
:1016A000352A74CF8B2D81538930D8F420E030E077
:1016B000C90103E0880F991F0A95E1F7220F331F34
:1016C000280F391F2B0D311D20533040F201089493
:1016D000411C511CB4908B2D80538A3048F32BABA6
:1016E0005ECF88E6B81619F494E0392A4FCFECE6BD
:1016F000BE1619F4F1E03F2A49CFBB83AA8323E643
:10170000B21639F41296BB83AA8312978C918E83FA
:1017100022C134E4B31639F044E6B41631F059E688
:10172000B516A9F502C081E0382A30FE08C014962B
:10173000BB83AA835E914E913E912E910AC0129670
:10174000BB83AA839E918E919C01442737FD4095CF
:10175000542F2EA73FA748AB59AB8EA59FA5A8A98C
:10176000B9A9BB238CF42EA53FA548A959A950952A
:101770004095309521953F4F4F4F5F4F2EA73FA784
:1017800048AB59AB8DE28983BAE02B2E80C03FE491
:10179000B31621F04FE6B41631F402C051E0352AF9
:1017A000A8E02A2E73C080E7B81689F41296BB838E
:1017B000AA839E918E919C0140E050E02EA73FA706
:1017C00048AB59AB30E4332AF8E7BF2E5DC043E79E
:1017D000B416D1F51296BB83AA83DE90CE90C114C5
:1017E000D10489F488E28E838EE68F8385E788872B
:1017F0008CE689878A8789E28B871C86E6E0CE2E75
:10180000D12CCC0EDD1E5AA957FD14C0452F5527EB
:1018100047FD509560E070E0C6010E947748009750
:1018200011F4FAA80EC0F82EFC188AA98F154CF4F2
:10183000F82E07C0F60101900020E9F73197FE2E3F
:10184000FC18198240E090C095E5B91621F0A5E793
:10185000BA1631F402C0B1E03B2A7AE0272E16C056
:10186000E8E5BE1621F0F8E7BF1609F070C033FEB8
:101870000BC02EA53FA548A959A921153105410541
:10188000510511F030E4332A60E1262E19824AA96D
:1018900047FD02C05FED35228EA59FA5A8A9B9A975
:1018A0000097A105B10549F49AA9992331F45EE2A4
:1018B000C52ED12CCC0EDD1E46C06EA47FA488A8F8
:1018C00099A84EE2C42ED12CCC0EDD1EE22CFF24B2
:1018D00000E010E06EA57FA588A999A9A80197014D
:1018E0000E94F14A6A3020F430E3A32EA60E08C00D
:1018F00027E5A22EA60EA8E5BA1611F4BFEDAB227D
:10190000F601A2926F016EA57FA588A999A9A801E9
:1019100097010E94F14A2EA73FA748AB59AB6E141E
:101920007F048006910618F039014A01D3CFF8E010
:101930002F1649F433FE07C020E3A21621F080E3FE
:10194000D6018E936D01FCA8FC184AA90DC0BB20DE
:1019500009F456C0BE82198296E0C92ED12CCC0E55
:10196000DD1E40E0FF24F394E42EEF18E7FCEE24A4
:101970008981882319F08F2D8F5F06C036FC02C045
:101980008F2D02C08F2D8E5FA82EAE0C032D10E080
:1019900080E3882E912C802291228114910421F4DD
:1019A0008BA98A190E94400A8981882329F061E065
:1019B00070E0CE01019609C006FF09C080E38C8368
:1019C000BD8262E070E0CE0104960E94610AB0E23E
:1019D0008B16910421F48BA98A190E94350A8E2D49
:1019E0000E94350A6F2D772767FD7095C6010E940A
:1019F000610A04FFABCD8BA98A190E94400AA6CDCB
:101A0000E5960FB6F894DEBF0FBECDBFDF91CF9144
:101A10001F910F91FF90EF90DF90CF90BF90AF900C
:101A20009F908F907F906F905F904F903F902F90FE
:101A300008952FB7F894909100019A3019F4529AB2
:101A40005A9802C03F9A479884B1886184B985B199
:101A5000877E85B99A3019F4529A5A9802C03F9AF3
:101A6000479884B58F7A84BD84B5836A84BD85B573
:101A7000877385BD85B5887F826085BD17BC88E783
:101A800088BD16BC80916E00897F80936E00809126
:101A90006E00816080936E002FBF08952091CE0468
:101AA0003091CF042F5F3F4F820F931F08952091F5
:101AB000CE043091CF04821B930B892F99278695F2
:101AC000807490E008951F920F920FB60F92112428
:101AD0002F933F934F935F936F937F938F939F9336
:101AE000AF93BF93EF93FF938091D5048150809380
:101AF000D5048F3FB9F489E08093D5048091060323
:101B00008F5F817080930603882319F481E08093AE
:101B1000D0048091CE049091CF0401969093CF048D
:101B20008093CE048091D3049091D404892BB1F09A
:101B30008091D3049091D40401979093D40480931E
:101B4000D3042091D3043091D40480910403909164
:101B5000050382239323892BD1F406C08FEF9FEFD7
:101B60009093050380930403809100018A3039F437
:101B700004C05A9A05C0479A03C05A9801C04798B2
:101B80008091B60883FF08C00E94EB3E05C080919B
:101B900000018A3081F7EDCFFF91EF91BF91AF91B6
:101BA0009F918F917F916F915F914F913F912F9175
:101BB0000F900FBE0F901F901895AC012091CE048E
:101BC0003091CF042F5F3F4F05C080917A00886C21
:101BD00080937A008091CE049091CF04B901681B64
:101BE000790BCB01840F951F80709078892F9927EE
:101BF0008695882351F30895AC012091CE0430914D
:101C0000CF042F5F3F4F8091CE049091CF04B90154
:101C1000681B790BCB01840F951F80709078892FFA
:101C200099278695882379F308959FB7F894579A52
:101C30005F9AE0EBF0E080818F7880838081836819
:101C40008083E1EBF0E08081867380838081866011
:101C500080838AE08093B3001092B200E0E7F0E066
:101C600080818A7F80838081826080839FBF089586
:101C70001F920F920FB60F921124FF920F931F9392
:101C80002F933F934F935F936F937F938F939F9384
:101C9000AF93BF93EF93FF9380910703815080939D
:101CA00007038F3F09F082C08091B0008093B0009D
:101CB0008091B00080688093B0008091930390E0A1
:101CC0009093D7048093D6048091E308F090D008D5
:101CD00080FF23C00091D6041091D70460911C05A9
:101CE00070911D0580911E0590911F0520E830E040
:101CF00040E050E00E94134BCA01B9012F2D30E0A3
:101D000040E050E00E949F4A20E032E040E050E096
:101D10000E94134B020F131F22C00091D604109192
:101D2000D70460911C0570911D0580911E0590914E
:101D30001F0520E830E040E050E00E94134BCA014C
:101D4000B9012F2D30E040E050E00E949F4A20E092
:101D500032E040E050E00E94134B021B130B109343
:101D6000D7040093D6042091D6043091D7048091F3
:101D7000D10890E02817390754F02091D60430910B
:101D8000D7048091D20890E08217930724F49093AF
:101D9000D7048093D6048091D6049091D704809381
:101DA000B3008091D3088093070306C08091B000F0
:101DB0008F738093B0005F98FF91EF91BF91AF91C7
:101DC0009F918F917F916F915F914F913F912F9153
:101DD0001F910F91FF900F900FBE0F901F901895BD
:101DE0009FB7F89411B812B88FEF80937E00ECE79C
:101DF000F0E080818F7180838081807E8083AAE77C
:101E0000B0E087E28C93EBE7F0E08081887F80830D
:101E10008C91886C8C939FBF08951F920F920FB680
:101E20000F921124EF92FF920F931F932F933F93E2
:101E30004F935F936F937F938F939F93AF93BF93D2
:101E4000CF93DF93EF93FF9380917A008773809312
:101E50007A008091F3048F5F8093F3048150853082
:101E600009F47EC0863090F4823009F440C083309B
:101E700030F48823F1F0813009F082C22FC0833022
:101E800009F441C0843009F07BC25AC0883009F49B
:101E9000B2C0893038F4863009F473C0873009F055
:101EA0006FC28CC0893009F4C3C08A3009F068C29F
:101EB000DBC180917800909179009093F204809337
:101EC000F10481E08093F4048091E8049091E904A6
:101ED00001969093E9048093E80456C280917800BB
:101EE000909179009093F0048093EF0482C08091E8
:101EF0007800909179009093EE048093ED0484E053
:101F00008093F40441C240910803509109038091E9
:101F10007800909179009A01220F331F240F351F0A
:101F200063E070E00E94CA4A260F371F3695279556
:101F300036952795309309032093080386E0E0CF78
:101F400080911605909117052091780030917900C5
:101F5000821B930B9093E1048093E00487E0D0CF41
:101F600080917800909179002091140530911505A9
:101F7000821B930B9093E3048093E2041092F40489
:101F800003C2809100012091F1043091F2048A3063
:101F900049F48091780090917900820F931F969573
:101FA000879506C08091780090917900820F931FE9
:101FB0009093DF048093DE0481E0A2CF8091000142
:101FC0002091EF043091F0048A3049F48091780038
:101FD00090917900820F931F9695879506C0809106
:101FE000780090917900820F931F9093DD04809385
:101FF000DC0482E085CF809100012091ED043091D6
:10200000EE048A3049F48091780090917900820F33
:10201000931F9695879506C08091780090917900DE
:10202000820F931F9093DB048093DA0485E068CFDE
:102030006091780070917900E0901805F090190592
:1020400000911A0510911B05882777FD8095982F20
:102050000E948449A80197010E9484480E94514926
:102060007093E5046093E404E091E404F091E504E6
:102070008091E2049091E304C091E004D091E104E6
:1020800097FF03C0909581959F4F64E070E00E9498
:10209000DE4A9B01CE01D7FF03C0909581959F4FEB
:1020A00064E070E00E94DE4A260F371FE20FF31F44
:1020B000F093E504E093E4048091E4049091E50456
:1020C00002970CF43EC0609118057091190580913B
:1020D0001A0590911B0520E030E84BE354E40E9480
:1020E000BF4988230CF078C06091180570911905DC
:1020F00080911A0590911B052AE037ED43EA5CE3D5
:102100000E948548609318057093190580931A05FD
:1021100090931B0580915C0590915D05845F9140D3
:1021200008F05AC0609118057091190580911A0540
:1021300090911B052DEC3CEC4CEC5DE30E94854836
:1021400043C08091E4049091E5048F5F9F4F0CF0B1
:1021500043C0609118057091190580911A059091FE
:102160001B0520E030E849E054E40E94C3491816FA
:102170009CF5609118057091190580911A05909150
:102180001B052AE037ED43EA5CE30E948448609334
:1021900018057093190580931A0590931B0580917B
:1021A0005C0590915D05845F9140B0F460911805E5
:1021B0007091190580911A0590911B052DEC3CEC4E
:1021C0004CEC5DE30E9484486093180570931905F8
:1021D00080931A0590931B05809178009091790067
:1021E0009093D9048093D80420914C0530914D05EB
:1021F00040914E0550914F058091E4049091E50483
:10220000AA2797FDA095BA2F820F931FA41FB51F71
:1022100080934C0590934D05A0934E05B0934F05C8
:10222000E0904C05F0904D0500914E0510914F0542
:1022300060914C0570914D0580914E0590914F0530
:1022400020E034E040E050E00E94134BE21AF30A31
:10225000040B150BE0924C05F0924D0500934E05D2
:1022600010934F0583E04CCEE0917800F091790017
:102270008091EA049091EB04E80FF91FF093EB04CE
:10228000E093EA048091EC048F5F8093EC04853046
:1022900008F476C0809178009091790090930F03B4
:1022A00080930E034091E6045091E7042091370893
:1022B000309138082E1B3F0B809184059091850545
:1022C000281B390B8091820390E0BC01269FC0013E
:1022D000279F900D369F900D11249A01A3E0220FA5
:1022E000331FAA95E1F7241B350B820F931F68E07B
:1022F00070E00E94DE4A7093E7046093E604E09089
:102300000A03F0900B0300910C0310910D03BF0121
:10231000882777FD8095982FA8019701220F331FFA
:10232000441F551F2E0D3F1D401F511F620F731F6D
:10233000841F951F24E030E040E050E00E94134BE2
:1023400020930A0330930B0340930C0350930D0327
:10235000209137083091380880910A0390910B033F
:10236000A0910C03B0910D03281B390B3093850508
:10237000209384051092EC041092EB041092EA046E
:102380001092F4041092F30480917C00807E90916E
:10239000F404892B80937C008091F304882329F036
:1023A00080917A00886C80937A00FF91EF91DF91A1
:1023B000CF91BF91AF919F918F917F916F915F91DD
:1023C0004F913F912F911F910F91FF90EF900F90A0
:1023D0000FBE0F901F9018951F93CF93DF9383E04C
:1023E0000E94913B182F853108F01A5017BD84E6E2
:1023F00090E00E94DD0D80910E0390910F038255B5
:102400009340C0F410E016C017BD82E390E00E9434
:10241000DD0DDF93CF931F920E94750A80910E030A
:1024200090910F030F900F900F908458934030F0CD
:102430001F5F02C0CDE8D1E01A3F30F3612F83E087
:102440000E949A3B109339088CE291E00E94DD0DC6
:10245000DF91CF911F910895EAE1F3E080E281934B
:1024600083E0EA36F807D1F708959F92AF92BF92C2
:10247000CF92DF92EF92FF920F931F93CF93DF9350
:102480008091F604282F30E0C90181709070682F88
:102490008823A9F08091F704882311F0815002C0AD
:1024A00080916A038093F704EAE1F3E080E281938C
:1024B00083E0EA36F807D1F78FEF8093BD04A901D6
:1024C0004270507021FF17C09091F70480916A0309
:1024D000981719F41092F70403C09F5F9093F704C4
:1024E000EAE1F3E080E2819393E0EA36F907D1F77D
:1024F0008FEF8093BD04662321F0452B11F01092DD
:10250000F7048091F704282F30E08A3040F481E10D
:102510008093F5043F932F9381E295E007C080E11B
:102520008093F5043F932F938CE195E09F938F93D5
:1025300081E08F930E94750A0F900F900F900F907B
:102540000F901091F704163009F4BDC2173090F4C3
:10255000123009F4D0C0133030F4112309F11130D6
:1025600009F05CC565C0143009F46FC1153008F07E
:10257000F0C117C1193009F457C31A3038F41730B5
:1025800009F4EFC2183009F049C510C31B3009F433
:10259000DDC31B3008F49CC31C3009F03FC528C4C0
:1025A0001092F5048CE095E09F938F9311E01F93B8
:1025B0000E94750A84E18093F50420910001822F26
:1025C0006AE00E94BE4A492F50E0822F0E94BE4A14
:1025D00090E02BE630E03F932F9325E430E03F93EB
:1025E0002F931F921F925F934F939F938F9387EF29
:1025F00094E09F938F931F930E94750A88E28093C3
:10260000F5040E94933D90E09F938F938AEE94E0AF
:102610009F938F931F930E94750A8CE38093F50418
:102620008AED94E09F938F931F930E94750ADCC3F9
:102630008091B60880FF47C01092F5048091840510
:10264000909185059F938F938BEC94E09F938F934C
:102650001F930E94750A84E18093F504809186059A
:10266000909187059F938F938CEB94E09F938F932A
:102670001F930E94750A88E28093F50480910E03EF
:1026800090910F039F938F938DEA94E09F938F9384
:102690001F930E94750A8CE38093F504809139089A
:1026A00090E09F938F938EE994E09F938F931F9375
:1026B0000E94750A8DB79EB744960FB6F8949EBFD8
:1026C0000FBE8DBFB0C484E18093F5048AE994E025
:1026D0009F938F931F930E94750A88E28093F5045D
:1026E0008BE894E09F938F931F930E94750A8DB798
:1026F0009EB70696E2CF1092F50482E894E09F938D
:102700008F9311E01F930E94750A84E18093F50472
:1027100060911C0570911D0580911E0590911F050B
:1027200020E034E040E050E00E94134B5F934F9371
:102730003F932F9384E794E09F938F931F930E947E
:10274000750A88E28093F50460912405709125054F
:10275000809126059091270520E034E040E050E08C
:102760000E94134B5F934F933F932F9385E694E022
:102770009F938F931F930E94750A8CE38093F504B7
:1027800080916E0390916F039F938F9386E594E001
:102790009F938F931F930E94750A8DB79EB746969D
:1027A0008CCF1092F50480914A0890914B082091AB
:1027B0004808309149089F938F933F932F9386E465
:1027C00094E09F938F9311E01F930E94750A84E118
:1027D0008093F50480914E0890914F0820914C0809
:1027E00030914D089F938F933F932F9386E394E00E
:1027F0009F938F931F930E94750A88E28093F5043C
:1028000080915208909153082091500830915108BE
:102810009F938F933F932F9386E294E09F938F93A0
:102820001F930E94750A8CE38093F50480915608EB
:102830009091570820915408309155089F938F9399
:102840003F932F9386E194E07BC01092F504E091D2
:10285000AF08F0E0EE0FFF1FEA5BF74F20813181F8
:10286000E091AE08F0E0EE0FFF1FEA5BF74F8081CA
:1028700091813F932F939F938F9386E094E09F9352
:102880008F9311E01F930E94750A84E18093F504F1
:10289000E091B108F0E0EE0FFF1FEA5BF74F2081F7
:1028A0003181E091B008F0E0EE0FFF1FEA5BF74FD7
:1028B000808191813F932F939F938F9386EF93E035
:1028C0009F938F931F930E94750A88E28093F5046B
:1028D000E091B308F0E0EE0FFF1FEA5BF74F2081B5
:1028E0003181E091B208F0E0EE0FFF1FEA5BF74F95
:1028F000808191813F932F939F938F9386EE93E0F6
:102900009F938F931F930E94750A8CE38093F50425
:10291000E091B508F0E0EE0FFF1FEA5BF74F208172
:102920003181E091B408F0E0EE0FFF1FEA5BF74F52
:10293000808191813F932F939F938F9386ED93E0B6
:102940009F938F931F930E94750A8DB79EB74C96E5
:10295000B4CE1092F50488EC93E09F938F9311E02E
:102960001F930E94750A0F900F900F9080910001A5
:102970008A3009F04AC084E18093F50440910A0549
:1029800050910B058091DA049091DB0420910A05A7
:1029900030910B05821B930B5F934F939F938F9303
:1029A00089EB93E09F938F931F930E94750A88E2AF
:1029B0008093F50440910C0550910D058091DC0445
:1029C0009091DD0420910C0530910D05821B930B35
:1029D0005F934F939F938F9389EA93E09F938F9395
:1029E0001F930E94750A8CE38093F50480910E0575
:1029F00090910F0520919B0830919C089F938F9395
:102A00003F932F9389E993E055C084E18093F504C7
:102A100080910A0590910B0562E070E00E94DE4A09
:102A20008091DA049091DB0420910A0530910B0526
:102A3000821B930B7F936F939F938F938AE893E00E
:102A40009F938F931F930E94750A88E28093F504E9
:102A500080910C0590910D0562E070E00E94DE4AC5
:102A60008091DC049091DD0420910C0530910D05DE
:102A7000821B930B7F936F939F938F938AE793E0CF
:102A80009F938F931F930E94750A8CE38093F504A4
:102A900080910E0590910F0562E070E00E94DE4A81
:102AA00080919B0890919C087F936F939F938F9345
:102AB0008AE693E09F938F931F930E94750A8DB7C8
:102AC0009EB74596FACD1092F5048DE593E09F935D
:102AD0008F9311E01F930E94750A84E18093F5049F
:102AE00080911405909115052091E2043091E30442
:102AF0009F938F933F932F938DE493E09F938F93B6
:102B00001F930E94750A88E28093F5048091160550
:102B1000909117052091E0043091E1049F938F93E9
:102B20003F932F938CE393E09F938F931F930E9487
:102B3000750A8CE38093F50460911805709119056E
:102B400080911A0590911B050E945149209191088E
:102B5000309192087F936F933F932F938BE293E092
:102B60003EC184E18093F5048091080390910903AC
:102B70009F938F938DE193E09F938F9311E01F9329
:102B80000E94750A88E28093F50480910305909174
:102B900004059F938F938FE093E09F938F931F93F0
:102BA0000E94750A8DB79EB70A9687CD1092F504DC
:102BB00080E093E09F938F9311E01F930E94750A2A
:102BC00084E18093F50480917003909171039F9349
:102BD0008F9381EF92E09F938F931F930E94750ACA
:102BE00088E28093F50480916E0390916F039F9328
:102BF0008F9382EE92E09F938F931F930E94750AAA
:102C00008CE38093F50480915005909151059F933A
:102C10008F9383ED92E09F938F931F930E94750A89
:102C20008DB79EB7429649CD1092F5048091660506
:102C30009091670520915E0530915F059F938F937A
:102C40003F932F9381EC92E09F938F9311E01F931A
:102C50000E94750A84E18093F50480916805909143
:102C6000690520916005309161059F938F933F9393
:102C70002F938FEA92E09F938F931F930E94750A80
:102C800088E28093F50480916A0590916B0520910C
:102C90006205309163059F938F933F932F938DE946
:102CA00092E09F938F931F930E94750A8CE3809309
:102CB000F50480916C0590916D052091640530912B
:102CC00065059F938F933F932F938BE892E038CEC7
:102CD0001092F50483E892E09F938F9311E01F9385
:102CE0000E94750A84E18093F5048091930390E03B
:102CF0009F938F9385E792E09F938F931F930E94FA
:102D0000750A88E28093F5048091D6049091D704E7
:102D10009F938F9387E692E09F938F931F930E94D8
:102D2000750A8CE38093F5042091D20830E08091FD
:102D3000D10890E03F932F939F938F9389E592E082
:102D40009F938F931F930E94750AB4CC1092F50441
:102D500089E492E09F938F9311E01F930E94750A7C
:102D600084E18093F50420915607332727FD3095A1
:102D700080915507992787FD90953F932F939F93B7
:102D80008F9389E392E09F938F931F930E94750A1C
:102D900088E28093F50420915707332727FD30956B
:102DA0008091580790E03F932F939F938F9389E2F0
:102DB00092E09F938F931F930E94750A8CE38093F8
:102DC000F50420915C0730E080915907992787FD31
:102DD00090953F932F939F938F9389E192E09F93D8
:102DE0008F931F930E94750A8DB79EB7489665CC46
:102DF00080917306882371F41092F5048CE092E0C0
:102E00009F938F9381E08F930E94750A0F900F908C
:102E10000F9009C120917506223071F02330B1F076
:102E2000809174062223E1F41092F50490E09F93C0
:102E30008F938BEF91E01BC01092F5048091740684
:102E400090E09F938F938AEE91E011C01092F50469
:102E50008091740690E09F938F9389ED91E007C075
:102E60001092F50490E09F938F9388EC91E09F93EC
:102E70008F9381E08F930E94750A0F900F900F90AF
:102E80000F900F90E0907606F0907706009178060C
:102E900010917906C801B70120E836E948E950E009
:102EA0000E94134B59016A01C801B70120E836E9B5
:102EB00048E950E00E94134B7B018C0120E137E28E
:102EC00040E050E00E94134BE90137FF03C0D0956A
:102ED000C195DF4FC801B70120E137E240E050E083
:102EE0000E94134B2AE030E040E050E00E94134B78
:102EF000B90137FF03C0709561957F4F84E18093DE
:102F0000F5047F936F93DF93CF93BF92AF9283EBE0
:102F100091E09F938F93992493949F920E94750AB6
:102F2000E0907A06F0907B0600917C0610917D0679
:102F3000C801B70120E836E948E950E00E94134B88
:102F400059016A01C801B70120E836E948E950E0B3
:102F50000E94134B7B018C0120E137E240E050E0FE
:102F60000E94134BE90137FF03C0D095C195DF4F95
:102F7000C801B70120E137E240E050E00E94134B66
:102F80002AE030E040E050E00E94134BB90137FFE7
:102F900003C0709561957F4F88E28093F5047F931D
:102FA0006F93DF93CF93BF92AF928EE991E09F939F
:102FB0008F939F920E94750AE0907E06F0907F06A4
:102FC0000091800610918106C801B70128EE33E018
:102FD00040E050E00E94134B59016A01C801B7015B
:102FE00028EE33E040E050E00E94134B9B0177FF56
:102FF00003C0309521953F4F8CE38093F5043F93B8
:103000002F93BF92AF928FE891E09F938F939F92FF
:103010000E94750A8DB79EB749964FCB11501093F9
:103020006A031092F7041092F604DF91CF911F917A
:103030000F91FF90EF90DF90CF90BF90AF909F9057
:10304000089587B18C6087B942984398089540915C
:10305000F8045091F9044431510500F14C3D5105FB
:10306000E8F42091FE043091FF04C901880F991FF4
:103070008417950710F4429A01C042982F5F3F4F82
:103080003093FF042093FE0421503040241735076D
:1030900030F01092FF041092FE0401C0429A409159
:1030A000FA045091FB044431510510F4439A0895F9
:1030B0004C3D5105E8F42091FC043091FD04C90118
:1030C000880F991F8417950710F4439A01C04398FD
:1030D0002F5F3F4F3093FD042093FC04215030407C
:1030E0002417350730F01092FD041092FC04089567
:1030F000439A08959FB7F8943998389A88B18360B5
:1031000088B9E9EBF0E080818C7F80838AE280934C
:10311000B8009FBF089585EA8093BC00089584E9B4
:103120008093BC0008958093BB0085E88093BC0029
:10313000089585EC8093BC00089585E88093BC00D9
:103140000895EF92FF920F931F938CEBE82EF12CD2
:1031500084E9F7018083109200050BEB10E0F80181
:103160008081809301051092010580E8F70180833A
:103170001092BD001092BA00F80110821092B900AE
:103180001092B8000E947A1885EAF7018083F8014E
:10319000108285E8F70180831F910F91FF90EF90D7
:1031A00008951F920F920FB60F9211248F939F9341
:1031B000EF93FF93809100058F5F8093000581500E
:1031C000833009F44AC0843028F4813091F0823091
:1031D000E0F50AC0853009F447C0853008F442C0E4
:1031E000863009F05DC04CC080910105880F8E5A71
:1031F0001AC0809101058F5F809301058150823054
:10320000C1F0833030F4882361F0813009F055C07B
:103210000DC08430A1F0843078F0853009F04DC0C5
:1032200011C080919D088093BB0026C080918808C2
:10323000FACF80919308F7CF8091A608F4CF8091C0
:103240009408F1CF8091AD08EECF809101058630D2
:1032500010F41092000585EA10C080910205880FD5
:103260008D5AE1CF85EC09C0E0910205F0E0809134
:10327000BB00E65CF74F808385E88093BC001DC0EF
:1032800080910205E82FF0E09091BB00E25CF74FDF
:1032900090838F5F80930205863010F010920205B4
:1032A00084E98093BC00109200058AE090E090933E
:1032B0006D0380936C0310920105FF91EF919F9134
:1032C0008F910F900FBE0F901F9018959FB7F89495
:1032D00056985E9A8AB180638AB98BB18F7C8BB91C
:1032E000809100018A3011F4539A5B98809180009C
:1032F0008C708093800080918100837E8093810018
:1033000080918100836C80938100809182008F7313
:103310008093820080916F00897F80936F008091FD
:103320006F00816280936F00109204051092030574
:103330009FBF08951F920F920FB60F9211242F93E3
:103340003F935F936F937F938F939F93AF93BF93BD
:1033500080910505882391F420910305309104059F
:10336000809103059091040568E070E00E94DE4AB8
:10337000261B370B30930405209303051092050597
:10338000BF91AF919F918F917F916F915F913F918D
:103390002F910F900FBE0F901F9018951F920F92B4
:1033A0000FB60F9211240F931F932F933F934F93B8
:1033B0005F936F937F938F939F93AF93BF93CF93BD
:1033C000DF93EF93FF9320918600309187008091E7
:1033D000060590910705281B390B80918600909176
:1033E00087009093070580930605C9018D5494408A
:1033F0000091080510910905835F9A4188F4043013
:1034000011053CF010926B03809105058F5F80934E
:10341000050581E090E0909309058093080598C028
:103420000E3011050CF094C0C9018B5F9040845B95
:10343000914008F072C0E901C25DD140F801EE0F81
:10344000FF1FEA5BF74F808191819E01281B390B9A
:10345000C90137FF03C0909581959F4F069784F46B
:103460008091030590910405883C91054CF480916E
:103470000305909104050A96909304058093030533
:10348000F801EE0FFF1FEA5BF74F20813181C90180
:10349000880F991F820F931F8C0F9D1F64E070E0AF
:1034A0000E94DE4A9B01CE010196861797071CF405
:1034B0002150304006C021976C177D0714F42F5F10
:1034C0003F4F8091030590910405E801CC0FDD1F6B
:1034D000833C9105BCF0FE01EA5BF74F808191814E
:1034E000A901481B590BCA0163E070E00E94DE4A43
:1034F000CB01880F991F860F971FCC59D74F9983FF
:10350000888304C0CC59D74F19821882F801EE0F76
:10351000FF1FEA5BF74F31832083F8013196F09368
:103520000905E0930805E530F10511F45D9A06C040
:103530005D98E630F10511F45C9A01C05C988091C9
:1035400000018A3029F4379711F45B9A01C05B9827
:103550008091030590910405892B49F08091030522
:103560009091040501979093040580930305FF91C2
:10357000EF91DF91CF91BF91AF919F918F917F910B
:103580006F915F914F913F912F911F910F910F90EC
:103590000FBE0F901F9018952F923F924F925F92FF
:1035A0006F927F928F929F92AF92BF92CF92DF9253
:1035B000EF92FF920F931F93CF93DF93CDB7DEB7B8
:1035C00022970FB6F894DEBF0FBECDBF80910E05D7
:1035D00090910F052091DE043091DF04821B930B44
:1035E00090939C0880939B088091DC049091DD046B
:1035F00020910C0530910D05821B930B90939A0836
:10360000809399088091DA049091DB0420910A0557
:1036100030910B05821B930B9093A5088093A4080F
:10362000E0908208F09083086091E2047091E304D6
:10363000882777FD8095982F2CE030E040E050E01F
:103640000E949F4A0027F7FC0095102FE60EF71EF8
:10365000081F191FC801B70122E030E040E050E028
:103660000E94134B3093830820938208E090A708B0
:10367000F090A8086091E0047091E104882777FD3C
:103680008095982F2CE030E040E050E00E949F4A67
:103690000027F7FC0095102FE60EF71E081F191FD4
:1036A000C801B70122E030E040E050E00E94134B37
:1036B0003093A8082093A708209191083091920890
:1036C0006091E4047091E504882777FD8095982F38
:1036D000442737FD4095542F620F731F841F951F99
:1036E00022E030E040E050E00E94134B309392081B
:1036F00020939108409144055091450560914605FD
:10370000709147052091E2043091E304C901880FCC
:10371000991F820F931F880F991F880F991FAA273F
:1037200097FDA095BA2F840F951FA61FB71F8093F2
:10373000440590934505A0934605B09347054091F5
:1037400048055091490560914A0570914B052091BB
:10375000E0043091E104C901880F991F820F931F83
:10376000880F991F880F991FAA2797FDA095BA2F38
:10377000840F951FA61FB71F809348059093490596
:10378000A0934A05B0934B052091E2043091E304E5
:103790008091540590915505820F931F9093550584
:1037A000809354052091E0043091E1048091560506
:1037B00090915705820F931F90935705809356055C
:1037C00080915805909159050196909359058093E1
:1037D0005805209140053091410540914205509196
:1037E000430580919B0890919C08AA2797FDA0957E
:1037F000BA2F820F931FA41FB51F8093400590938B
:103800004105A0934205B093430580919B08909198
:103810009C089C01442737FD4095542F80919E08B9
:1038200090919F08A091A008B091A108280F391F7E
:103830004A1F5B1F20939E0830939F084093A00867
:103840005093A108203B83E8380788E0480780E0D0
:10385000580764F0205B33484840504020939E084E
:1038600030939F084093A0085093A10880919E0830
:1038700090919F08A091A008B091A108B7FF0CC03B
:1038800080559C47A74FBF4F80939E0890939F08F9
:10389000A093A008B093A10890918C059A839923D6
:1038A00009F08AC080918D05882309F085C0809138
:1038B000B60886FF81C060919B0870919C0820919A
:1038C0003005309131054091320550913305E0903B
:1038D0009503FF2400E010E0882777FD8095982F5E
:1038E0000E949F4A20E038E040E050E00E94134BE5
:1038F000CA01B901A80197010E949F4A20E030E166
:1039000040E050E00E94134B59016A012093CB051F
:103910003093CC054093CD055093CE0560919B0824
:1039200070919C08209138053091390540913A05F5
:1039300050913B05882777FD8095982F0E949F4ADC
:1039400020E038E040E050E00E94134BCA01B9018A
:10395000A80197010E949F4A20E030E140E050E03A
:103960000E94134B2093C7053093C8054093C905A7
:103970005093CA05D601C501D7FE07C0B095A095E2
:10398000909581959F4FAF4FBF4F81389105A1050D
:10399000B10574F457FF07C05095409530952195B7
:1039A0003F4F4F4F5F4F2138310541055105A4F07E
:1039B00081E08093530510C01092C7051092C8058E
:1039C0001092C9051092CA051092CB051092CC0531
:1039D0001092CD051092CE058091990890919A0889
:1039E0002090CB053090CC054090CD055090CE0571
:1039F000820D931D90939A088093990800919908DD
:103A000010919A08A090C705B090C805C090C9054C
:103A1000D090CA0580919603682E77248824992433
:103A2000C401B301A60195010E949F4A20E032E043
:103A300040E050E00E94134B020F131F10939A08AE
:103A40000093990820913C0530913D0540913E0539
:103A500050913F058091990890919A08AA2797FD67
:103A6000A095BA2F820F931FA41FB51F80933C050A
:103A700090933D05A0933E05B0933F0540913805D6
:103A80005091390560913A0570913B0580919908F4
:103A900090919A082091880530918905821B930B9B
:103AA000AA2797FDA095BA2F840F951FA61FB71FB1
:103AB0008093380590933905A0933A05B0933B0560
:103AC0008091380590913905A0913A05B0913B0558
:103AD000E0907803F090790300917A0310917B03D2
:103AE000E816F9060A071B0704F580E197E2A0E053
:103AF000B0E08E199F09A00BB10B8093380590930D
:103B00003905A0933A05B0933B0580913805909113
:103B10003905A0913A05B0913B0580933C059093FF
:103B20003D05A0933E05B0933F05209138053091A7
:103B3000390540913A0550913B0588279927DC01CA
:103B40008E199F09A00BB10B281739074A075B078D
:103B500004F580EF98EDAFEFBFEFE80EF91E0A1FF6
:103B60001B1FE0923805F092390500933A05109337
:103B70003B058091380590913905A0913A05B091A7
:103B80003B0580933C0590933D05A0933E05B09383
:103B90003F058091DC049091DD040F9734F488E1B7
:103BA0009CEF90939A08809399088091DC049091FF
:103BB000DD04079734F480E398EF90939A0880939C
:103BC00099089091000199839A30A9F48091DC04BE
:103BD0009091DD04835F934034F088EE93E09093FE
:103BE0009A08809399088091DC049091DD048A5FA3
:103BF0009340DCF014C08091DC049091DD04855E7C
:103C0000974034F088EE93E090939A088093990857
:103C10008091DC049091DD04835F974034F080ED67
:103C200097E090939A08809399088091A4089091C6
:103C3000A5088A199B099093A5088093A408009170
:103C4000A4081091A508C401B301A20191010E942A
:103C50009F4A20E032E040E050E00E94134B021BFC
:103C6000130B1093A5080093A408209134053091FC
:103C7000350540913605509137058091A408909103
:103C8000A508AA2797FDA095BA2F820F931FA41FFE
:103C9000B51F8093340590933505A0933605B093F6
:103CA0003705409130055091310560913205709192
:103CB00033058091A4089091A50820918A05309140
:103CC0008B05821B930BAA2797FDA095BA2F840F13
:103CD000951FA61FB71F8093300590933105A093C1
:103CE0003205B09333058091300590913105A09154
:103CF0003205B0913305E0907403F09075030091A4
:103D0000760310917703E816F9060A071B0704F5F6
:103D100088EA91E6A0E0B0E08E199F09A00BB10BF4
:103D20008093300590933105A0933205B09333050D
:103D30008091300590913105A0913205B091330505
:103D40008093340590933505A0933605B0933705DD
:103D50002091300530913105409132055091330565
:103D600088279927DC018E199F09A00BB10B281712
:103D700039074A075B0704F588E59EE9AFEFBFEF17
:103D8000E80EF91E0A1F1B1FE0923005F092310564
:103D900000933205109333058091300590913105E1
:103DA000A0913205B0913305809334059093350589
:103DB000A0933605B09337058091DA049091DB0427
:103DC0000F9734F488E19CEF9093A5088093A408A2
:103DD0008091DA049091DB04079734F480E398EF44
:103DE0009093A5088093A40899819A30A9F48091B2
:103DF000DA049091DB04835F934034F088EE93E023
:103E00009093A5088093A4088091DA049091DB0434
:103E10008A5F9340DCF014C08091DA049091DB0457
:103E2000855E974034F088EE93E09093A5088093E8
:103E3000A4088091DA049091DB04835F974034F00A
:103E400080ED97E09093A5088093A40880917A0074
:103E5000886C80937A008091400590914105A091F3
:103E60004205B091430580932C0590932D05A093B6
:103E70002E05B0932F058091300590913105A091CA
:103E80003205B091330580931C0590931D05A093D6
:103E90001E05B0931F058091380590913905A091BA
:103EA0003A05B0913B058093240590932505A09396
:103EB0002605B09327058091340590913505A09192
:103EC0003605B09137058093200590932105A09386
:103ED0002205B093230580913C0590913D05A0916A
:103EE0003E05B0913F058093280590932905A09346
:103EF0002A05B0932B058091B60887FF63C02A81FD
:103F0000222309F05FC080918D05882309F05AC0F3
:103F10008091A4089091A508893C91055CF02091BE
:103F2000A4083091A5088091A4089091A50820527A
:103F3000334011C08091A4089091A50888539F4FE9
:103F4000A4F42091A4083091A5088091A408909130
:103F5000A508205E3C4F880F991F880F991F280FD6
:103F6000391F3093A5082093A40880919908909157
:103F70009A08893C91055CF02091990830919A0843
:103F80008091990890919A082052334011C08091F5
:103F9000990890919A0888539F4FA4F4209199080A
:103FA00030919A088091990890919A08205E3C4F30
:103FB000880F991F880F991F280F391F30939A086F
:103FC0002093990822960FB6F894DEBF0FBECDBF9E
:103FD000DF91CF911F910F91FF90EF90DF90CF90E5
:103FE000BF90AF909F908F907F906F905F904F9019
:103FF0003F902F9008950F931F930AE710E0F80168
:104000008081877380838091DA049091DB049093A0
:10401000A5088093A4088091DC049091DD0490931E
:104020009A08809399088091DE049091DF04909320
:104030009C0880939B086091E2047091E3048827B8
:1040400077FD8095982F2CE030E040E050E00E9412
:104050009F4A70938308609382086091E004709196
:10406000E104882777FD8095982F0E949F4A7093DE
:10407000A8086093A7088091E4049091E5049093C8
:10408000920880939108F8018081886C8083609108
:10409000D90870E080E090E024EC39E040E050E0A6
:1040A0000E949F4A60937403709375038093760314
:1040B000909377036091DA0870E080E090E00E94CE
:1040C0009F4A609378037093790380937A03909367
:1040D0007B031F910F910895809103059091040532
:1040E000813A91050CF40AC38091B9088B3F98F08E
:1040F0008B3F19F480915E050EC08C3F19F48091BE
:10410000600509C08D3F19F48091620504C08E3F9F
:1041100021F4809164058093830380918303882335
:1041200019F41092830304C08F3F11F4809383032A
:104130008091B8088B3F98F08B3F19F480915E0511
:104140000EC08C3F19F48091600509C08D3F19F4B1
:104150008091620504C08E3F21F4809164058093B4
:10416000820380918203882319F41092820305C090
:10417000843618F084E6809382038091BA088B3FDE
:1041800098F08B3F19F480915E050EC08C3F19F4B6
:104190008091600509C08D3F19F48091620504C0CB
:1041A0008E3F21F480916405809384038091840381
:1041B000882319F41092840305C0843618F084E62D
:1041C000809384038091BC088B3F98F08B3F19F457
:1041D00080915E050EC08C3F19F48091600509C086
:1041E0008D3F19F48091620504C08E3F21F48091C7
:1041F00064058093850380918503882319F41092C8
:10420000850304C08F3F11F4809385038091C30818
:104210008B3F98F08B3F19F480915E050EC08C3F68
:1042200019F48091600509C08D3F19F480916205F1
:1042300004C08E3F21F480916405809386038091B1
:104240008603882319F41092860304C08F3F11F46B
:10425000809386038091C4088B3F98F08B3F19F4BC
:1042600080915E050EC08C3F19F48091600509C0F5
:104270008D3F19F48091620504C08E3F21F4809136
:10428000640580938703809187038B3010F48AE064
:1042900002C08F3F11F4809387038091C5088B3F44
:1042A00098F08B3F19F480915E050EC08C3F19F495
:1042B0008091600509C08D3F19F48091620504C0AA
:1042C0008E3F21F480916405809388038091880358
:1042D000882319F41092880304C08F3F11F480934F
:1042E00088038091CA088B3F98F08B3F19F4809126
:1042F0005E050EC08C3F19F48091600509C08D3FAA
:1043000019F48091620504C08E3F21F48091640508
:1043100080938A0380918A03882319F410928A0378
:1043200004C08F3F11F480938A038091CB088B3FA8
:1043300098F08B3F19F480915E050EC08C3F19F404
:104340008091600509C08D3F19F48091620504C019
:104350008E3F21F48091640580938B0380918B03C1
:10436000882319F410928B0304C08F3F11F48093BB
:104370008B038091CC088B3F98F08B3F19F4809190
:104380005E050EC08C3F19F48091600509C08D3F19
:1043900019F48091620504C08E3F21F48091640578
:1043A00080938C0380918C03882319F410928C03E2
:1043B00004C08F3F11F480938C038091CD088B3F14
:1043C00098F08B3F19F480915E050EC08C3F19F474
:1043D0008091600509C08D3F19F48091620504C089
:1043E0008E3F21F48091640580938D0380918D032D
:1043F000882319F410928D0304C08F3F11F4809329
:104400008D038091CE088B3F98F08B3F19F48091FB
:104410005E050EC08C3F19F48091600509C08D3F88
:1044200019F48091620504C08E3F21F480916405E7
:1044300080938E0380918E03882319F410928E034B
:1044400004C08F3F11F480938E038091DE088B3F70
:1044500098F08B3F19F480915E050EC08C3F19F4E3
:104460008091600509C08D3F19F48091620504C0F8
:104470008E3F21F48091640580938F0380918F0398
:10448000882319F410928F0304C08F3F11F4809396
:104490008F038091DF088B3F98F08B3F19F4809158
:1044A0005E050EC08C3F19F48091600509C08D3FF8
:1044B00019F48091620504C08E3F21F48091640557
:1044C0008093900380919003882319F410929003B5
:1044D00004C08F3F11F4809390038091E0088B3FDC
:1044E00098F08B3F19F480915E050EC08C3F19F453
:1044F0008091600509C08D3F19F48091620504C068
:104500008E3F21F480916405809391038091910303
:10451000882319F41092910304C08F3F11F4809303
:1045200091038091E1088B3F98F08B3F19F48091C3
:104530005E050EC08C3F19F48091600509C08D3F67
:1045400019F48091620504C08E3F21F480916405C6
:104550008093920380919203882319F4109292031E
:1045600004C08F3F11F4809392038091CF088B3F5A
:1045700098F08B3F19F480915E050EC08C3F19F4C2
:104580008091600509C08D3F19F48091620504C0D7
:104590008E3F21F48091640580939303809193036F
:1045A000882319F41092930304C08F3F11F4809371
:1045B00093038091D4088B3F98F08B3F19F480913E
:1045C0005E050EC08C3F19F48091600509C08D3FD7
:1045D00019F48091620504C08E3F21F48091640536
:1045E0008093940380919403882319F41092940388
:1045F00004C08F3F11F4809394038091D7088B3FC0
:1046000098F08B3F19F480915E050EC08C3F19F431
:104610008091600509C08D3F19F48091620504C046
:104620008E3F21F4809164058093950380919503DA
:10463000882319F41092950304C08F3F11F48093DE
:1046400095038091D8088B3F98F08B3F19F48091A7
:104650005E050EC08C3F19F48091600509C08D3F46
:1046600019F48091620504C08E3F21F480916405A5
:104670008093960380919603882319F410929603F1
:1046800004C08F3F11F4809396038091DD088B3F27
:1046900098F08B3F19F480915E050EC08C3F19F4A1
:1046A0008091600509C08D3F19F48091620504C0B6
:1046B0008E3F21F480916405809397038091970346
:1046C000882319F41092970304C08F3F11F480934C
:1046D000970360918A0370E080E090E00E94D746E3
:1046E00027E137EB41ED58E30E943C4A60937E039B
:1046F00070937F038093800390938103089580914A
:104700005A05882361F51092A60810929D08109210
:10471000880810929308109294081092AD08809126
:10472000C004882331F0809393088091930880938C
:104730009D088091C104882331F08093880880917E
:1047400088088093A6088091C204882311F0809382
:10475000AD088091C304882311F0809394081092CF
:104760000005109201050E948B18089510921505FE
:1047700010921405109217051092160580E090E033
:10478000A0E0B0E08093180590931905A0931A0556
:10479000B0931B0510920B0510920A0510920D059F
:1047A00010920C0510920F0510920E0510929503B1
:1047B000109296030E94FB1F84E690E00E94DD0D9C
:1047C0000E94FB1F8091B60880FF10C080910E03ED
:1047D00090910F03875B934038F480910E03909182
:1047E0000F038E5E924010F40E94EC118091DA0467
:1047F0009091DB0490930B0580930A058091DC0473
:104800009091DD0490930D0580930C058091DE045A
:104810009091DF0490930F0580930E0580910C0515
:1048200090910D05909311058093100580910A05D4
:1048300090910B05909313058093120584E00E94DC
:10484000A23B8050944058F18091A7089091A8080D
:1048500097FF03C0909581959F4F6CE070E00E9498
:10486000DE4A709317056093160580918208909137
:10487000830897FF03C0909581959F4F6CE070E08F
:104880000E94DE4A70931505609314056091D80468
:104890007091D904882777FD8095982F17C084E000
:1048A0000E94A23B909315058093140586E00E9418
:1048B000A23B909317058093160588E00E94A23BC7
:1048C000AA2797FDA095BA2FBC01CD010E9484496B
:1048D000609318057093190580931A0590931B0532
:1048E0001092300510923105109232051092330566
:1048F0001092340510923505109236051092370546
:10490000109238051092390510923A0510923B0525
:1049100010923C0510923D0510923E0510923F0505
:1049200010924005109241051092420510924305E5
:104930001092A5081092A40810929A081092990853
:1049400010929C0810929B0880910A0390910B038F
:10495000A0910C03B0910D03909338088093370811
:104960001092E7041092E60410924C0510924D0547
:1049700010924E0510924F0580916E0390916F0337
:10498000909371038093700382E390E09093D4043A
:104990008093D3046091D90870E080E090E024EC2B
:1049A00039E040E050E00E949F4A6856754C8F4FB6
:1049B0009F4F609374037093750380937603909375
:1049C00077036091DA0870E080E090E00E949F4AEF
:1049D0006856754C8F4F9F4F60937803709379039F
:1049E00080937A0390937B0310927D0310927C0353
:1049F000109277051092760510927905109278053D
:104A000060916E0370916F03882777FD8095982FD2
:104A10002EE036E040E050E00E949F4A60939E08FE
:104A200070939F088093A0089093A1081092A30808
:104A30001092A20808951F93182F0EC080915A0556
:104A4000882361F484E690E09093D4048093D304A7
:104A50008AEF90E00E94FC0D115080F71F9108959D
:104A60008091AE08E82FF0E0EE0FFF1FEA5BF74FF2
:104A7000808191818D5E9F4F14F010929803808108
:104A800091818A5B9F4FDCF4809198038823B9F46D
:104A900081E080939803809152058F5F8093520547
:104AA00080915205853028F4809152050E941B2583
:104AB000089588EE93E09093D4048093D3040895EE
:104AC0002F923F924F925F926F927F928F929F921E
:104AD000AF92BF92CF92DF92EF92FF920F931F930C
:104AE000CF93DF93CDB7DEB7A2970FB6F894DEBFB2
:104AF0000FBECDBF0E94CC1A299A20917405309127
:104B000075058091C008482F50E0465F5F4F5A8777
:104B100049874217530714F43A8729878091030580
:104B200090910405883791050CF073C080910301C2
:104B3000882399F480910403909105038F5F9F4F20
:104B400061F488E99AE39093D4048093D30480E0DD
:104B50009CE090930503809304038091B1059091AC
:104B6000B205009731F001979093B2058093B1059B
:104B700004C010925A0510925B05809100018A30A2
:104B800011F4289A01C0289880915C0590915D05E8
:104B9000895E9340D8F18091C708A82FB0E0BA870A
:104BA000A98781E080935B05E091AE082E2F30E06D
:104BB000220F331FF901EC59F74F11821082A09197
:104BC000AF08B0E0AA0FBB1FFD01EC59F74F1182EF
:104BD0001082E091B1084E2F50E0440F551FCA01DA
:104BE0008C59974FFC01118210822A5B374FF901D3
:104BF00011821082AA5BB74F11961C921E924A5BDB
:104C0000574FDA0111961C921E92DAC310925A0580
:104C1000D7C380910305909104058D3891050CF45C
:104C2000CFC310925B058091C80822E3829FC00128
:104C300011249093B2058093B105E985FA85B9975F
:104C40006CF080915C0590915D05FFEF8F3F9F07B1
:104C500029F0019690935D0580935C0580915C0539
:104C600090915D058F3F910509F0E8F41092C3051E
:104C70001092C4051092C5051092C6051092BF058A
:104C80001092C0051092C1051092C20510927305D2
:104C9000109272058A3F910531F481E090E0909383
:104CA000A9058093A80520915E0530915F0580914C
:104CB000B208E82FF0E0EE0FFF1FEA5BF74F8081AC
:104CC000918182599F4F281739071CF42F5F3F4F5E
:104CD0000CC08081918182599F4F821793074CF4B9
:104CE0002115310531F02150304030935F0520937C
:104CF0005E0520916005309161058091B308E82F31
:104D0000F0E0EE0FFF1FEA5BF74F8081918182593F
:104D10009F4F281739071CF42F5F3F4F0CC080812D
:104D2000918182599F4F821793074CF421153105C9
:104D300031F021503040309361052093600520917F
:104D40006205309163058091B408E82FF0E0EE0F22
:104D5000FF1FEA5BF74F8081918182599F4F28178F
:104D600039071CF42F5F3F4F0CC08081918182591D
:104D70009F4F821793074CF42115310531F02150D4
:104D80003040309363052093620520916405309193
:104D900065058091B508E82FF0E0EE0FFF1FEA5B94
:104DA000F74F8081918182599F4F281739071CF452
:104DB0002F5F3F4F0CC08081918182599F4F821796
:104DC00093074CF42115310531F0215030403093D8
:104DD00065052093640520916605309167058091F3
:104DE00058089091590882599F4F281739071CF489
:104DF0002F5F3F4F0EC080915808909159088259FB
:104E00009F4F821793074CF42115310531F0215043
:104E100030403093670520936605209168053091F6
:104E2000690580915A0890915B0882599F4F281715
:104E300039071CF42F5F3F4F0EC080915A089091A4
:104E40005B0882599F4F821793074CF42115310557
:104E500031F021503040309369052093680520914E
:104E60006A0530916B0580915C0890915D088259CC
:104E70009F4F281739071CF42F5F3F4F0EC08091BA
:104E80005C0890915D0882599F4F821793074CF4FC
:104E90002115310531F02150304030936B052093BE
:104EA0006A0520916C0530916D0580915E089091A6
:104EB0005F0882599F4F281739071CF42F5F3F4F17
:104EC0000EC080915E0890915F0882599F4F8217B3
:104ED00093074CF42115310531F0215030403093C7
:104EE0006D0520936C0580915E0590915F0597FF9D
:104EF00005C010925F0510925E050AC08F3F9105B4
:104F000039F034F08FEF90E090935F0580935E0569
:104F1000809160059091610597FF05C01092610531
:104F2000109260050AC08F3F910539F034F08FEF81
:104F300090E0909361058093600580916205909167
:104F4000630597FF05C010926305109262050AC0C1
:104F50008F3F910539F034F08FEF90E09093630527
:104F600080936205809164059091650597FF05C067
:104F700010926505109264050AC08F3F910539F0C3
:104F800034F08FEF90E090936505809364058091F5
:104F900066059091670597FF05C01092670510920E
:104FA00066050AC08F3F910539F034F08FEF90E02D
:104FB00090936705809366058091680590916905D7
:104FC00097FF05C010926905109268050AC08F3FCF
:104FD000910539F034F08FEF90E09093690580935C
:104FE000680580916A0590916B0597FF05C0109246
:104FF0006B0510926A050AC08F3F910539F034F0B5
:105000008FEF90E090936B0580936A0580916C051B
:1050100090916D0597FF05C010926D0510926C057B
:105020000AC08F3F910539F034F08FEF90E09093F4
:105030006D0580936C05E091B008F0E0EE0FFF1F66
:10504000EA5BF74F80819181813591050CF40EC1A7
:1050500080915A05882309F009C18091B108E82F91
:10506000F0E0EE0FFF1FEA5BF74F808191818C34F7
:1050700091050CF4BFC08091B0058F5F8093B0059F
:10508000893C08F4F3C01092B005299810925D0590
:1050900010925C058091AE08282F30E0D901AA0F4C
:1050A000BB1FAA5BB74F8D919C91119787349105D7
:1050B0009CF48091AF08E82FF0E0EE0FFF1FEA5B51
:1050C000F74F8081918197FF03C0909581959F4F05
:1050D000873491050CF46BC08091AF08682F70E0A5
:1050E000DB01AA0FBB1FAA5BB74F8D919C91119753
:1050F000873491053CF0F901EE0FFF1FEA5BF74F93
:10510000808191818D919C918734910564F0F901A2
:10511000EE0FFF1FEA5BF74F808191818734910585
:1051200014F042E001C041E0FB01EE0FFF1FEA5B1B
:10513000F74F80819181863491055CF4F901EE0F7F
:10514000FF1FEA5BF74F80819181873491050CF056
:1051500043E0FB01EE0FFF1FEA5BF74F8081918177
:105160008A5B9F4F5CF4F901EE0FFF1FEA5BF74F7C
:1051700080819181873491050CF044E0660F771FA0
:105180006A5B774FDB018D919C918A5B9F4F5CF44A
:10519000220F331F2A5B374FF901808191818634BA
:1051A00091050CF445E0842F0E94B23B1CC0809115
:1051B000B60883FF18C08081918197FF03C0909546
:1051C00081959F4F44977CF48D919C918A5B9F4F72
:1051D00054F481E08093520588EE93E09093D404D8
:1051E0008093D30443C00E94933D0E94D03B0E9411
:1051F000B62335C080819181855B9F4FACF580914E
:10520000B0058F5F8093B005893C80F11092B005A6
:1052100029986FEF7FEF84E00E94AA3B10925D0512
:1052200010925C050E94B6236091140570911505DB
:1052300084E00E94AA3B609116057091170586E0F4
:105240000E94AA3B609118057091190580911A057A
:1052500090911B050E94564988E00E94AA3B0E943B
:10526000933D0E941B2502C01092B005E091B0084A
:10527000F0E0EE0FFF1FEA5BF74F808191818B5AC0
:105280009F4F0CF09DC0E091B108F0E0EE0FFF1FC2
:10529000EA5BF74F80819181855B9F4F0CF06AC07C
:1052A0008091AF058F5F8093AF05893C08F464C09F
:1052B0001092AF0581E090E090935D0580935C05CE
:1052C00081E080935A051092BB051092BC051092A4
:1052D000BD051092BE051092400510924105109236
:1052E000420510924305109230051092310510923C
:1052F000320510923305109238051092390510923C
:105300003A0510923B0580911C0590911D05A091D6
:105310001E05B0911F058093340590933505A09329
:105320003605B09337058091240590912505A0910D
:105330002605B091270580933C0590933D05A093E9
:105340003E05B0933F051092C3051092C40510921C
:10535000C5051092C6051092BF051092C0051092A7
:10536000C1051092C2058091B60885FF05C00E9454
:10537000C64002C01092AF05E091B108F0E0EE0F18
:10538000FF1FEA5BF74F808191818C349105B4F067
:105390008091AE058F5F8093AE05893C88F01092B6
:1053A000AE0510925D0510925C0510925A05809131
:1053B000B60885FF05C00E944C4102C01092AE05A0
:1053C00080916B03815080936B0380916B038F3FBF
:1053D00029F080915B05882309F477C30E946C2033
:1053E00060916E0570916F057AA369A38091AE08F4
:1053F000E82EFF24D701AA0FBB1FCD018A5B974F70
:10540000FC018081918198A38F8F8091BD08682EC7
:105410007724AC59B74F0D90BC91A02DBE8FAD8FA6
:105420008091BE08A82EBB24209176053091770587
:105430003C8F2B8F20907005309071058091AF08C4
:10544000082F10E0C801880F991FDC01AA5BB74F35
:105450000D90BC91A02DBA8FA98F8C59974FDC016C
:105460008D919C91988F8F8BE0917805F0917905C3
:10547000FE8BED8BE091B108AE2FB0E0AA0FBB1F01
:10548000AA5BB74F0D90BC91A02DBC8BAB8BE0916C
:10549000B008F0E0EE0FFF1FEA5BF74FC080D1804D
:1054A00028E730E0C20ED31ED0927505C092740575
:1054B0006091870370E080E090E00E94D74620E092
:1054C00030E040E251E40E94854820E030E040E8CE
:1054D0005CE30E943C4A6F87788B898B9A8B609340
:1054E000A9087093AA088093AB089093AC086091C8
:1054F000880370E080E090E00E94D74620E030EE24
:105500004BE256E40E94E948609395087093960830
:1055100080939708909398082091C504222331F036
:105520008AE090E09093D4048093D304E22F22FF8A
:1055300009C080919203482F50E0440F551F440F3B
:10554000551F10C023FD03C040E050E00BC0809108
:10555000920390E0880F991F880F991F44275527C1
:10556000481B590B20917E0530917F05C901B3E09E
:10557000880F991FBA95E1F7821B930B840F951F33
:1055800068E070E00E94DE4A2B0170937F05609313
:105590007E05E4FF09C080919203482F50E0440F3C
:1055A000551F440F551F10C0E5FD03C040E050E0FB
:1055B0000BC08091920390E0880F991F880F991F6C
:1055C00044275527481B590B8091800590918105F0
:1055D0009C01E3E0220F331FEA95E1F7281B390B0A
:1055E000CA01820F931F68E070E00E94DE4A4B01FF
:1055F00070938105609380058091C404282F83FFF8
:1056000003C082E390E004C082FF07C08EEC9FEFEE
:10561000909383058093820504C0109283051092B5
:10562000820521FF09C080917C0390917D03019642
:1056300090937D0380937C0324FF09C080917C03B9
:1056400090917D03019790937D0380937C034F8D10
:1056500058A1469DC001479D900D569D900D112467
:1056600029A13AA1220F331F69A17AA1260F371F62
:10567000ED8DFE8DEA9DD001EB9DB00DFA9DB00D34
:1056800011244B8D5C8DA41BB50BBAA3A9A3820F6B
:10569000931F64E070E00E94DE4A89A19AA1860F00
:1056A000971F9AA389A3C20162E070E00E94DE4ABC
:1056B000A9A1BAA1A60FB71FBAA3A9A3B0936F055A
:1056C000A0936E05E98DFA8DE69DC001E79D900DD2
:1056D000F69D900D11249101220F331F220D331DD1
:1056E0004F89588DB501469F5001479FB00C569F7A
:1056F000B00C1124AD89BE89AA1ABB0A820F931F70
:1057000064E070E00E94DE4AA60EB71EC40162E0AB
:1057100070E00E94DE4AA60EB71EB0927105A092FC
:1057200070052091820530918305220F331F220FCF
:10573000331FEB89FC892E1B3F0B3093730520939D
:10574000720580915C0780FF56C08091920381387A
:1057500008F451C080915507992787FD9095AC01B9
:10576000469DC001479D900D569D900D112469A145
:105770007AA1680F791F70936F0560936E05809111
:105780005607992787FD9095DC01A69DC001A79D2E
:10579000900DB69D900D1124A80EB91EB092710502
:1057A000A092700580915707992787FD9095280F43
:1057B000391F30937305209372052091BB0830E0A8
:1057C00080915907992787FD9095FC012E9FC00174
:1057D0002F9F900D3E9F900D112490937D038093F9
:1057E0007C038091580790E08C159D0524F49093DC
:1057F000750580937405809174059091750597FFE8
:1058000004C010927505109274058091B60882FF4D
:105810000CC080E090E0A0E0B0E080939508909309
:105820009608A0939708B093980820E030E040E0F5
:1058300050E06F85788989899A890E94BF498823B9
:1058400064F480E090E0A0E0B0E08093A908909339
:10585000AA08A093AB08B093AC0820E030E040E089
:1058600050E060919508709196088091970890910A
:1058700098080E94BF49882364F480E090E0A0E08B
:10588000B0E08093950890939608A0939708B09302
:105890009808E0916E05F0916F0520917A0530919E
:1058A0007B05CF0164E070E00E94DE4A77FF03C011
:1058B000709561957F4F261737077CF4CF01F7FF6E
:1058C00003C0909581959F4F64E070E00E94DE4A8E
:1058D00070937B0560937A0506C021503040309369
:1058E0007B0520937A05E0917005F0917105209178
:1058F0007C0530917D05CF0164E070E00E94DE4AB6
:1059000077FF03C0709561957F4F261737077CF4AA
:10591000CF01F7FF03C0909581959F4F64E070E041
:105920000E94DE4A70937D0560937C0506C021507D
:10593000304030937D0520937C05F801EE0FFF1F6A
:10594000EA5BF74F208131818091D508482F50E0E4
:105950004217530744F48091E20882FF04C081E0BB
:1059600080938E0515C080918E05882389F0F801FB
:10597000EE0FFF1FEA5BF74F208131818091D6083F
:10598000BA01681B71092617370714F410928E05A7
:10599000F801EE0FFF1FEA5BF74F808191816627C8
:1059A0007727641B750B8617970744F48091E208EC
:1059B00083FF04C081E080938F0515C080918F051F
:1059C000882389F0000F111F0A5B174FD8012D9112
:1059D0003C918091D60890E0841B950B8217930729
:1059E00014F410928F05F701EE0FFF1FEA5BF74FDB
:1059F000808191814817590744F48091E20880FF23
:105A000004C081E08093910515C0809191058823A1
:105A100089F0F701EE0FFF1FEA5BF74F208131811C
:105A20008091D608FA01E81BF1092E173F0714F4FC
:105A300010929105F701EE0FFF1FEA5BF74F80818F
:105A400091818617970744F48091E20881FF04C092
:105A500081E08093900517C080919005882399F08C
:105A6000EE0CFF1C26E438E0E20EF31ED7012D9168
:105A70003C918091D60890E0841B950B8217930788
:105A800014F41092900580918E05882321F4809162
:105A90008F05882321F081E080938D0502C010924C
:105AA0008D0580919105882321F4809190058823AC
:105AB00051F081E080938C0510928D0510928E0537
:105AC00010928F0502C010928C0580918D0588235D
:105AD00021F480918C05882351F08091D40890E0C6
:105AE000E985FA858E179F0714F49A878987809134
:105AF000910390E09093F9048093F80480919203CD
:105B000090E09093FB048093FA040E942718809100
:105B10005B05882381F11092730510927205109233
:105B20006F0510926E05109271051092700580E05D
:105B300090E0A8ECBFE38093A9089093AA08A093F3
:105B4000AB08B093AC088BE09CEBA2E3BCE3809382
:105B5000950890939608A0939708B0939808109290
:105B60008D0510928C0510927B0510927A0510928B
:105B70007D0510927C052091840830918508409124
:105B800086085091870880911C0590911D05A09171
:105B90001E05B0911F05820F931FA41FB51F809390
:105BA000840890938508A0938608B0938708209175
:105BB0008B0830918C0840918D0850918E0880910F
:105BC000240590912505A0912605B0912705820F07
:105BD000931FA41FB51F80938B0890938C08A093EC
:105BE0008D08B0938E0850908C05552029F4809133
:105BF0008D05882309F44FC01092E9041092E8043F
:105C000010924405109245051092460510924705E2
:105C1000109248051092490510924A0510924B05C2
:105C200010928408109285081092860810928708B6
:105C300010928B0810928C0810928D0810928E088A
:105C40008091300590913105A0913205B0913305D6
:105C50008093340590933505A0933605B0933705AE
:105C60008091380590913905A0913A05B0913B0596
:105C700080933C0590933D05A0933E05B0933F056E
:105C800010928B0510928A05109289051092880552
:105C9000552009F0F5C080918D05882309F0F0C0EA
:105CA00060911C0570911D0580911E0590911F0546
:105CB000A090C208BB24CC24DD24E0908208F090A0
:105CC0008308A60195010E94134B0027F7FC00955D
:105CD000102F2E193F09400B510BCA01B90120E1C9
:105CE00030E040E050E00E94134B39014A016091DE
:105CF0002405709125058091260590912705E09057
:105D0000A708F090A808A60195010E94134B002750
:105D1000F7FC0095102F2E193F09400B510BCA01BB
:105D2000B90120E130E040E050E00E94134B7901DE
:105D30008A0180917A0590917B05819734F4809156
:105D40007C0590917D058197A4F0C401B30123E007
:105D500030E040E050E00E94134B39014A01C80195
:105D6000B70123E030E040E050E00E94134B79019E
:105D70008A01E091B108F0E0EE0FFF1FEA5BF74FF8
:105D80000190F081E02DF7FF03C0F095E195FF4F02
:105D90007A97A4F0C401B30123E030E040E050E082
:105DA0000E94134B39014A01C801B70123E030E0DA
:105DB00040E050E00E94134B79018A01F1E26F1636
:105DC00071048104910434F070E2672E712C812CEF
:105DD000912C11C020EE62162FEF72062FEF820673
:105DE0002FEF920644F460EE662E6FEF762E6FEF83
:105DF000862E6FEF962E31E2E316F10401051105B0
:105E000034F050E2E52EF12C012D112D11C040EEA1
:105E1000E4164FEFF4064FEF04074FEF140744F476
:105E200040EEE42E4FEFF42E4FEF042F4FEF142FE0
:105E30008091300590913105A0913205B0913305E4
:105E400086199709A809B9098093300590933105FF
:105E5000A0933205B09333058091380590913905B0
:105E6000A0913A05B0913B058E199F09A00BB10B8B
:105E70008093380590933905A0933A05B0933B057C
:105E80008091E8049091E9048F3F910509F008F4AE
:105E900045C4552009F0DCC380918D05882309F0A5
:105EA000D7C380915305882309F0D2C36091840839
:105EB00070918508809186089091870820E031E0F4
:105EC00040E050E00E94134B2093840830938508F3
:105ED000409386085093870860918B0870918C08D6
:105EE00080918D0890918E0820E031E040E050E0F4
:105EF0000E94134B20938B0830938C0840938D089D
:105F000050938E08E090C208FF2400E010E020913A
:105F10004405309145054091460550914705C8011B
:105F2000B7010E949F4A20E031E040E050E00E942B
:105F3000134B2093440530934505409346055093F9
:105F40004705209148053091490540914A055091F7
:105F50004B05C801B7010E949F4A20E031E040E0B4
:105F600050E00E94134B209348053093490540931D
:105F70004A0550934B056091840870918508809183
:105F800086089091870820914405309145054091FD
:105F9000460550914705E090DB08FF2400E010E043
:105FA000621B730B840B950BA80197010E94134B86
:105FB000CA01B90120E031E040E050E00E94134BFB
:105FC000690130938B0520938A0560918B0870914D
:105FD0008C0880918D0890918E0820914805309111
:105FE000490540914A0550914B05621B730B840B88
:105FF000950BA80197010E94134BCA01B90120E03B
:1060000031E040E050E00E94134B89013093890554
:106010002093880580917A0590917B058197BCF447
:1060200080917C0590917D0581978CF4E091B10879
:10603000F0E0EE0FFF1FEA5BF74F0190F081E02DDB
:10604000F7FF03C0F095E195FF4F7A9794F0C601F2
:1060500062E070E00E94DE4A70938B0560938A05CF
:10606000C80162E070E00E94DE4A70938905609387
:106070008805E0902005F0902105009122051091FF
:10608000230580911C0590911D05A0911E05B091DE
:106090001F05E81AF90A0A0B1B0BE092B705F092EC
:1060A000B8050093B9051093BA0580913405909115
:1060B0003505A0913605B09137058E199F09A00BC3
:1060C000B10B8093340590933505A0933605B093BA
:1060D0003705609028057090290580902A059090DA
:1060E0002B058091240590912505A0912605B0915E
:1060F0002705681A790A8A0A9B0A6092B30570928A
:10610000B4058092B5059092B60580913C059091BA
:106110003D05A0913E05B0913F0586199709A80954
:10612000B90980933C0590933D05A0933E05B0933B
:106130003F052091A2083091A308213831054CF089
:1061400080910E0590910F05019690930F05809315
:106150000E0520583F4F4CF480910E0590910F058D
:10616000019790930F0580930E051092A30810924B
:10617000A20881E090E090939F0580939E05109285
:10618000A4051092A5051092A6051092A70580916E
:10619000840890918508A0918608B0918708209185
:1061A0009605309197054091980550919905281BC7
:1061B000390B4A0B5B0B57FF07C050954095309544
:1061C00021953F4F4F4F5F4F20523E44404050403B
:1061D0000CF0C1C071E0E71670E1F70670E0070748
:1061E00070E017070CF452C080919D05882309F4D4
:1061F00049C0D801C7012CE0B595A795979587951B
:106200002A95D1F7019690939F0580939E05D8011A
:10621000C701F3E0B595A79597958795FA95D1F7BE
:106220008093A4059093A505A093A605B093A70518
:1062300089589341A040B04064F088E893E1A0E021
:10624000B0E08093A4059093A505A093A605B09314
:10625000A7056091A4057091A5058091A605909170
:10626000A70520E031E040E050E00E94134B809110
:106270008A0590918B05820F931F90938B058093D5
:106280008A0566C081E080939D0562C010929D05DD
:10629000F0E0EF16F0EFFF06FFEF0F07FFEF1F072D
:1062A0000CF056C080919C05882309F44DC08827C6
:1062B0009927DC018E199F09A00BB10BECE0B59575
:1062C000A79597958795EA95D1F7019690939F05A5
:1062D00080939E05C801B70128E030E040E050E01F
:1062E0000E94134B2093A4053093A5054093A60567
:1062F0005093A70528573C4E4F4F5F4F64F488E7F3
:106300009CEEAFEFBFEF8093A4059093A505A093FB
:10631000A605B093A7056091A4057091A50580918D
:10632000A6059091A70520E031E040E050E00E94F2
:10633000134B80918A0590918B05820F931F909348
:106340008B0580938A0511C081E080939C050DC068
:1063500010929C050AC010929F0510929E0584EF32
:1063600091E090937303809372038091DC08C82EB0
:10637000DD2480919E0590919F05C816D90624F4CE
:10638000D0929F05C0929E0571E0E71674E0F70673
:1063900070E0070770E0170774F080910A0590918C
:1063A0000B0520919E0530919F05820F931F9093BE
:1063B0000B0580930A0580E0E8168CEFF8068FEF56
:1063C00008078FEF180774F480910A0590910B0568
:1063D00020919E0530919F05821B930B90930B0596
:1063E00080930A0581E090E090939F0580939E053D
:1063F0001092A0051092A1051092A2051092A3057B
:1064000080918B0890918C08A0918D08B0918E0896
:1064100020919205309193054091940550919505F6
:10642000281B390B4A0B5B0B57FF07C05095409553
:10643000309521953F4F4F4F5F4F20523E44404093
:1064400050400CF0C1C0A1E06A16A0E17A06A0E0BD
:106450008A06A0E09A060CF452C080919B0588231E
:1064600009F449C0D401C3017CE0B595A79597957F
:1064700087957A95D1F7019690939F0580939E0515
:10648000D401C30163E0B595A795979587956A9563
:10649000D1F78093A0059093A105A093A205B09396
:1064A000A30589589341A040B04064F088E893E187
:1064B000A0E0B0E08093A0059093A105A093A20571
:1064C000B093A3056091A0057091A1058091A205EC
:1064D0009091A30520E031E040E050E00E94134B92
:1064E0008091880590918905820F931F909389056B
:1064F0008093880566C081E080939B0562C01092FE
:106500009B05F0E06F16F0EF7F06FFEF8F06FFEFC1
:106510009F060CF056C080919A05882309F44DC05F
:1065200088279927DC0186199709A809B9095CE031
:10653000B595A795979587955A95D1F7019690931C
:106540009F0580939E05C401B30128E030E040E040
:1065500050E00E94134B2093A0053093A105409377
:10656000A2055093A30528573C4E4F4F5F4F64F44C
:1065700088E79CEEAFEFBFEF8093A0059093A10555
:10658000A093A205B093A3056091A0057091A10509
:106590008091A2059091A30520E031E040E050E019
:1065A0000E94134B8091880590918905820F931F5B
:1065B000909389058093880511C081E080939A05A6
:1065C0000DC010929A050AC010929F0510929E0568
:1065D00084EF91E0909373038093720380919E0502
:1065E00090919F05C816D90624F4D0929F05C092B9
:1065F0009E0571E0671674E0770670E0870670E02C
:10660000970674F080910C0590910D0520919E05E0
:1066100030919F05820F931F90930D0580930C0579
:1066200080E068168CEF78068FEF88068FEF98066B
:10663000CCF480910C0590910D0520919E05309130
:106640009F05821B930B90930D0580930C050AC048
:10665000109289051092880510928B0510928A0578
:106660001092530520E030E040E050E06091950842
:106670007091960880919708909198080E94BF4960
:10668000882341F4109289051092880510928B0599
:1066900010928A058091840890918508A0918608BF
:1066A000B09187088093960590939705A0939805DD
:1066B000B093990580918B0890918C08A0918D08DA
:1066C000B0918E088093920590939305A0939405C2
:1066D000B093950510924405109245051092460519
:1066E00010924705109248051092490510924A05EC
:1066F00010924B051092840810928508109286081B
:106700001092870810928B0810928C0810928D08B6
:1067100010928E081092E9041092E804C09072055D
:10672000D09073058601D7FE04C0002711270C19ED
:106730001D0900311105C4F08091B60884FD14C014
:1067400081E090E09093A9058093A80580919E0830
:1067500090919F0890937103809370038AEF90E06B
:106760009093730380937203E090BF08B60188276B
:1067700077FD8095982F2E2D30E040E050E00E946C
:106780009F4A9801442737FD4095542F0E949F4A05
:1067900020E032E040E050E00E94134B89019A0172
:1067A000FF24EC9CC001ED9C900DFC9C900D1124ED
:1067B00064E070E00E94DE4A600F711F882777FD59
:1067C0008095982F6093BB057093BC058093BD05A1
:1067D0009093BE05209140053091410540914205BE
:1067E00050914305261B370B480B590B209340054E
:1067F00030934105409342055093430580914005F5
:1068000090914105A0914205B09143058155934C6B
:10681000A040B04064F080E593ECA0E0B0E080934D
:10682000400590934105A0934205B09343058091A4
:10683000400590914105A0914205B0914305805BD0
:106840009C43AF4FBF4F64F480EB9CE3AFEFBFEFCF
:106850008093400590934105A0934205B093430572
:106860008091B60883FF5AC180915205882339F080
:1068700080915A05882319F40E9430254FC16091F8
:106880001C0570911D0580911E0590911F0520E04B
:1068900032E040E050E00E94134B890137FF03C013
:1068A000109501951F4F60912405709125058091E9
:1068B00026059091270520E032E040E050E00E945C
:1068C000134B690137FF04C0D094C194D108D3940D
:1068D000C016D1060CF4680129E1C216D10444F5B2
:1068E0008091A8059091A905892B11F180917203DF
:1068F00090917303892BE1F488EC90E09093D40499
:106900008093D30460919E0870919F088091A008A5
:106910009091A1082EE036E040E050E00E94134B39
:1069200030937103209370031092A9051092A8056B
:1069300080916E0390916F0397FF03C020E030E0D9
:1069400029C0E0906E03F0906F034CE152E0E40E3A
:10695000F51E0027F7FC0095102F60919E0870919E
:106960009F088091A0089091A1082EE036E040E0B9
:1069700050E00E94134BE21AF30A040B150BC801F6
:10698000B70128E631E040E050E00E94134B9B0144
:10699000245B3040C60168E070E00E94DE4A6F5F11
:1069A0007F4FC90143E0880F991F4A95E1F70E9484
:1069B000DE4A3B01882477FC8094982C80919E08C5
:1069C00090919F08A091A008B091A108680E791E2F
:1069D0008A1E9B1E60929E0870929F088092A0085B
:1069E0009092A10880918603A82EBB24CA9CC00166
:1069F000CB9C900DDA9C900D112460E470E00E9415
:106A0000DE4A2501461A570A141415040CF080C0FA
:106A10008091720390917303009711F001977AC0EF
:106A20008091A2089091A308820F931F9093A308CE
:106A30008093A20880917C0590917D0520917A0534
:106A400030917B05820F931F68E070E00E94DE4A60
:106A50006B0160E470E0C60ED71E809170039091C8
:106A60007103AA2797FDA095BA2F0CE1E02E02E052
:106A7000F02E012D112DE81AF90A0A0B1B0BC40187
:106A8000B3012EE036E040E050E00E94134BE20EEE
:106A9000F31E041F151FC801B70128E631E040E0CE
:106AA00050E00E94134B645B7040649DC001659D83
:106AB000900D749D900D1124B6010E94DE4AC5010F
:106AC000880F991F8A0D9B1D8617970734F09095A4
:106AD00081959F4F681779070CF4BC012091400500
:106AE000309141054091420550914305CB01AA27C1
:106AF00097FDA095BA2F820F931FA41FB51F8093F7
:106B0000400590934105A0934205B093430506C00C
:106B10008AEF90E090937303809372038091B6089C
:106B200085FF17C080918C038093D40580918F03DB
:106B30008093D305809190038093D50580915B0568
:106B4000882311F086EE02C0809162050E943A44CB
:106B500008C0109277051092760510927905109270
:106B600078058091AA0581508093AA058F3F09F08E
:106B7000B4C088E18093AA0560911C0570911D0541
:106B800080911E0590911F05E090C208FF2400E04F
:106B900010E0A80197010E94134B309360072093E7
:106BA0005F076091240570912505809126059091DD
:106BB0002705A80197010E94134B30936207209389
:106BC0006107809182089091830890936407809375
:106BD00063078091A7089091A80890936607809317
:106BE000650780919B0890919C089093680780931B
:106BF0006707809184059091850590936A0780933B
:106C0000690760914C0570914D0580914E059091FA
:106C10004F0520E032E040E050E00E94134B3093FB
:106C20006C0720936B078091030590910405909366
:106C3000700780936F0780910803909109039093E8
:106C400072078093710780919D0890E0909374077C
:106C5000809373078091930890E0909376078093D8
:106C600075078091A60890E0909378078093770746
:106C70008091880890E090937A07809379078091BB
:106C8000AD0890E090937C0780937B0780919408F7
:106C900090E090937E0780937D078091910890917A
:106CA00092089093800780937F078091D6049091FB
:106CB000D7049093880780938707809176059091F9
:106CC000770590939C0780939B078091780590911E
:106CD000790590939E0780939D0780918C0588236A
:106CE000A9F06091A4087091A508882777FD809588
:106CF000982F0E9484492091A9083091AA084091B8
:106D0000AB085091AC080E943C4A32C060911C050F
:106D100070911D0580911E0590911F05E090A408BB
:106D2000F090A5080E94844920919508309196081A
:106D300040919708509198080E943C4A5B016C0171
:106D40000027F7FC0095102FC801B7010E94844965
:106D50002091A9083091AA084091AB085091AC0845
:106D60000E943C4A9B01AC01C601B5010E948548C6
:106D70000E9451497093A5086093A40880918D05E5
:106D80008823A9F06091990870919A08882777FD67
:106D90008095982F0E9484492091A9083091AA08D3
:106DA0004091AB085091AC080E943C4A32C06091BF
:106DB0002405709125058091260590912705E09086
:106DC0009908F0909A080E94844920919508309182
:106DD000960840919708509198080E943C4A5B01A0
:106DE0006C010027F7FC0095102FC801B7010E9425
:106DF00084492091A9083091AA084091AB0850918C
:106E0000AC080E943C4A9B01AC01C601B5010E943E
:106E100085480E94514970939A086093990860913F
:106E20009B0870919C08A0902C05B0902D05C090F7
:106E30002E05D0902F058091950890919608A091ED
:106E40009708B091980889839A83AB83BC8388277D
:106E500077FD8095982F0E9484497B018C01609179
:106E6000A9087091AA088091AB089091AC089B0189
:106E7000AC010E9485489B01AC01C801B7010E948A
:106E80003C4A7B018C01C601B5010E9484492981DD
:106E90003A814B815C810E943C4A20E030E040E036
:106EA0005FE30E943C4A9B01AC01C801B7010E940C
:106EB00085480E94514970939C0860939B0880917B
:106EC000A4089091A50890938A07809389078091E0
:106ED000990890919A0890938C0780938B078091E2
:106EE000A4089091A5088150904434F080E090E48B
:106EF0009093A5088093A4088091A4089091A50878
:106F00008050904C34F480E090EC9093A5088093EE
:106F1000A4088091990890919A088150904434F087
:106F200080E090E490939A08809399088091990862
:106F300090919A088050904C34F480E090EC9093BB
:106F40009A088093990880919B0890919C088150A1
:106F5000904434F080E090E490939C0880939B08E8
:106F600080919B0890919C088050904C34F480E074
:106F700090EC90939C0880939B08A984BA84AA0CF7
:106F8000BB1CAA0CBB1C8091B608282F80FFC7C071
:106F900080915B05882309F0C2C08091830321FFA3
:106FA0000EC0823310F58091840590918505449739
:106FB00090938705809386051092AD0519C02091A6
:106FC0007C0330917D03280F311D8091BB0890E038
:106FD000AC01249FC001259F900D349F900D11247A
:106FE0004497909387058093860581E08093AD0553
:106FF0002091840530918505409186055091870543
:10700000421753070CF08BC08091AD05882309F41B
:1070100086C08091840390E0241B350BBC01629FE5
:10702000C001639F900D729F900D112464E070E089
:107030000E94DE4A4B01C090E604D090E7046091C4
:107040004C0570914D0580914E0590914F05E09053
:107050008503FF2400E010E020E830E040E050E04D
:107060000E94134BC801B7010E949F4A20E230E002
:1070700040E050E00E94134B7EEF283E370714F4A7
:1070800028EE3EEF8091AB059091AC05FC01A4E0A9
:10709000EE0FFF1FAA95E1F7E81BF90BC60162E0AE
:1070A00070E00E94DE4AE61BF70B81E029313807C9
:1070B00014F028E131E0E21BF30BC50188199909AE
:1070C0008E0F9F1F60E170E00E94DE4A7093AC0556
:1070D0006093AB058091B70890E0880F991F880FE7
:1070E000991F6817790764F4A816B9062CF09093D5
:1070F000AC058093AB0504C0B092AC05A092AB0583
:107100008091AB059091AC05A816B90624F4B09215
:10711000AC05A092AB05A090AB05B090AC058091FA
:10712000C108882E99248401000F111F000F111F20
:10713000C80180559040BAA2A9A28A159B0514F4F3
:107140009AA389A3A9A1BAA1B0936E07A0936D07D2
:1071500020919B0830919C088091BB059091BC05C3
:10716000A091BD05B091BE0542E0880F991FAA1FEE
:10717000BB1F4A95D1F7281B390BE9A1FAA1E13AC7
:10718000F105ACF0F595E7952E173F070CF4F901E2
:1071900089A19AA162E070E00E94DE4A7095619533
:1071A0007F4FCF01E617F7076CF4CB010BC0C90185
:1071B000205B3F4F14F480EB9FEF8135910514F075
:1071C00080E590E0980149A15AA1241B350B2817AE
:1071D00039070CF4C90129A13AA1201B310B2C015C
:1071E000821793070CF429018091A4089091A508B7
:1071F00060906E0570906F058619970990939008BE
:1072000080938F0820E030E040E050E069817A818F
:107210008B819C810E94BF498823F1F1E0901C057D
:10722000F0901D0500911E0510911F056091C3058A
:107230007091C4058091C5059091C6050E9484494E
:107240005B016C01C801B7010E94844929813A8120
:107250004B815C810E943C4A7B018C01B3018827F1
:1072600077FD8095982F0E9484499B01AC01C8014D
:10727000B7010E9484489B01AC01C601B5010E9480
:1072800085480E9451496093C3057093C40580935B
:10729000C5059093C6051CC020918F0830919008B9
:1072A000442737FD4095542F8091C3059091C40524
:1072B000A091C505B091C605820F931FA41FB51FED
:1072C0008093C3059093C405A093C505B093C605EC
:1072D0008091C3059091C405A091C505B091C605E4
:1072E00081509A4FA040B04064F080E09AEFA0E057
:1072F000B0E08093C3059093C405A093C505B093F7
:10730000C6058091C3059091C405A091C505B091B3
:10731000C60580509640AF4FBF4F64F480E096E0C2
:10732000AFEFBFEF8093C3059093C405A093C5054D
:10733000B093C60560918F087091900880917E038C
:1073400090917F03A0918003B09181038B879C87EC
:10735000AD87BE87882777FD8095982F0E94844946
:107360007B018C016091C3057091C4058091C505B6
:107370009091C6050E9484499B01AC016B857C8578
:107380008D859E850E943C4A9B01AC01C801B701D6
:107390000E9485480E9451497B018C016B01C2010A
:1073A00057FE04C0882799278419950962E070E088
:1073B0000E94DE4AA9A1BAA16A0F7B1F882777FD28
:1073C0008095982F2091970330E040E050E00E9494
:1073D0009F4A20E430E040E050E00E94134B3E839F
:1073E0002D83C216D3060CF497012D803E80309475
:1073F00021943108339438872F832215330514F4F0
:1074000038862F828091990890919A086090700533
:10741000709071058619970990938A08809389085E
:1074200020E030E040E050E069817A818B819C81EE
:107430000E94BF498823F1F1E0902405F0902505D2
:1074400000912605109127056091BF057091C00538
:107450008091C1059091C2050E9484495B016C0135
:10746000C801B7010E94844929813A814B815C811E
:107470000E943C4A7B018C01B301882777FD8095EF
:10748000982F0E9484499B01AC01C801B7010E945A
:1074900084489B01AC01C601B5010E9485480E9449
:1074A00051496093BF057093C0058093C1059093C7
:1074B000C2051CC02091890830918A08442737FDF5
:1074C0004095542F8091BF059091C005A091C105B2
:1074D000B091C205820F931FA41FB51F8093BF05F3
:1074E0009093C005A093C105B093C2058091BF05DC
:1074F0009091C005A091C105B091C20581509A4FED
:10750000A040B04064F080E09AEFA0E0B0E080934B
:10751000BF059093C005A093C105B093C2058091AB
:10752000BF059091C005A091C105B091C2058050E2
:107530009640AF4FBF4F64F480E096E0AFEFBFEFEF
:107540008093BF059093C005A093C105B093C20579
:107550006091890870918A08882777FD8095982F17
:107560000E9484497B018C016091BF057091C00528
:107570008091C1059091C2050E9484499B01AC0194
:107580006B857C858D859E850E943C4A9B01AC0164
:10759000C801B7010E9485480E9451492D813E8152
:1075A000621773070CF49B018101221633060CF459
:1075B00089012F81388549A15AA1240F351FC8019F
:1075C00062E070E00E94DE4A7B01C901860F971FCE
:1075D0008419950964E070E00E94DE4A86169706D9
:1075E00014F4B40107C08091C00890E068177907CF
:1075F0000CF4BC0160939D08240D351DC9018E1942
:107600009F0964E070E00E94DE4A8616970614F433
:10761000B40107C08091C00890E0681779070CF4A6
:10762000BC016093930829A13AA16F817885261B3C
:10763000370BC701820F931F8419950964E070E02E
:107640000E94DE4A8616970614F4B40107C08091A2
:10765000C00890E0681779070CF4BC016093A60895
:10766000240D351DC9018E199F0964E070E00E9448
:10767000DE4A8616970614F4B40107C08091C0084C
:1076800090E0681779070CF4BC016093880889A121
:107690009AA1840D951D800F911F64E070E00E94F7
:1076A000DE4A8616970614F4B40107C08091C0081C
:1076B00090E0681779070CF4BC016093AD0889A1CC
:1076C0009AA1801B910B9AA389A38419950964E060
:1076D00070E00E94DE4A8616970644F08091C0084A
:1076E00090E04B01681779070CF44C0180929408E4
:1076F000A2960FB6F894DEBF0FBECDBFDF91CF913B
:107700001F910F91FF90EF90DF90CF90BF90AF90BF
:107710009F908F907F906F905F904F903F902F90B1
:107720000895A0E0B0E0A80FB11D0E94654B802D28
:1077300090E00895A0E0B0E0A80FB11D062E0E94D1
:10774000774B0895A0E0B0E0A80FB11D0E94724BE6
:10775000CF010895A0E0B0E0A80FB11D0B010E9479
:10776000834B0895863008F085E0A2E0B0E0082E53
:107770000E94774B0895982F863008F095E086E4B4
:10778000989FD0011124AC59BF4FEEEAF8E0182EB3
:107790000E94884BA2E0B0E0092E0E94774B08952A
:1077A000982F863008F095E086E4989FD001112448
:1077B000AC59BF4FEEEAF8E0182E0E946D4B0895C9
:1077C00081E08093AE0882E08093AF0843E040936D
:1077D000B00864E06093B10855E05093B20836E019
:1077E0003093B30887E08093B40828E02093B5086D
:1077F00088EE8093B6089EE19093B7088BEF809354
:10780000B9088AE08093BA089093B8089093BC08AE
:107810004093BB082093BD0840E14093BE083093DD
:10782000BF082093C00886EE8093C1089093C208D9
:1078300080E88093C30834E63093C40888E78093D7
:10784000C5088EE58093C60883E28093C70884E16B
:107850008093C8081092C9084093CA088DEF80939E
:10786000CB083093CC089AE59093CD089093CE083E
:107870009093DE089093DF081092E0081092E108E0
:107880003093CF0888E28093D0081092E30822E377
:107890002093D10886E98093D2085093D30820938F
:1078A000D4089093D5082093D6081092E2089093BC
:1078B000D7085093D8083093D9083093DA0880E27B
:1078C0008093DB086093DC082093DD08A8EEB8E025
:1078D000E9E9F3E089E001900D928150E1F7089524
:1078E00081E08093AE0882E08093AF0843E040934C
:1078F000B00864E06093B10855E05093B20836E0F8
:107900003093B30887E08093B40828E02093B5084B
:1079100088E68093B6089EE19093B7088BEF80933A
:10792000B9088AE08093BA089093B8089093BC088D
:107930004093BB088CE08093BD0880E18093BE0833
:107940003093BF082093C00886EE8093C1089093BF
:10795000C20880E88093C30880E58093C40888E764
:107960008093C5088EE58093C60883E28093C7089C
:107970009093C8081092C90840E24093CA088DEF5E
:107980008093CB0834E63093CC082AE52093CD08C9
:107990002093CE082093DE082093DF081092E008A1
:1079A0001092E1083093CF0888E28093D0081092BB
:1079B000E30892E39093D10886E98093D20850932C
:1079C000D3089093D4082093D5089093D6081092AA
:1079D000E2082093D7085093D8083093D908309301
:1079E000DA084093DB086093DC088BE48093DD08C1
:1079F000A8EEB8E0E3EAF3E087E001900D92815051
:107A0000E1F7089581E08093AE0882E08093AF08AB
:107A100083E08093B00854E05093B10835E0309390
:107A2000B20886E08093B30887E08093B40828E02A
:107A30002093B50888E68093B6089EE19093B70836
:107A40008BEF8093B9088AE08093BA089093B808C6
:107A50009093BC085093BB088FE08093BD0890932F
:107A6000BE088CE08093BF082093C00886EE809308
:107A7000C1089093C20880E88093C30880E5809392
:107A8000C40846E94093C5088EE58093C60883E2A2
:107A90008093C7089093C8081092C90880E2809329
:107AA000CA088DEF8093CB0824E62093CC089AE592
:107AB0009093CD089093CE089093DE089093DF08C2
:107AC0001092E0081092E1082093CF0888E280939A
:107AD000D0081092E30882E38093D1084093D20843
:107AE0003093D3088093D4089093D5088093D60818
:107AF0001092E2089093D7083093D8082093D908C1
:107B00002093DA0880E18093DB085093DC0820930F
:107B1000DD08A8EEB8E0EBEAF3E086E001900D9214
:107B20008150E1F7089522E030E0D9010E94654BD1
:107B3000802D863028F082E0D901082E0E94774BF4
:107B400090E008950F931F93CF93DF93A1E0B0E0EF
:107B50000E94654B802D863469F18FE395E09F93F9
:107B60008F931F920E94750A0E94023DC0E0D0E0F0
:107B70000F900F900F900C2FC23039F0C33019F4D2
:107B80000E94E03B04C0C43010F00E94703C802F83
:107B90000E94BB3B2196C630D10569F7A2E0B0E058
:107BA00083E0082E0E94774BA1E0B0E086E4082E27
:107BB0000E94774B02E010E0D8010E94654B802DB7
:107BC0000E94D03BD8010E94654B802D90E09F938E
:107BD0008F9386E295E09F938F931F920E94750A80
:107BE0000F900F900F900F900F90DF91CF911F91FA
:107BF0000F910895CF93DF93DC01EC01EA81FB81C3
:107C000021918E81815019F48981E81BF109ED01E0
:107C1000FB83EA838E839FB7F8948C9181508C9379
:107C20009FBF822F90E0DF91CF910895FC011082D9
:107C30007583648373836283418347834683089596
:107C4000CF93DF93DC019C91ED018981981718F0A7
:107C500080E090E016C0ED01EC81FD8161938F81A1
:107C6000815019F48981E81BF109ED018F83FD83AF
:107C7000EC839FB7F8948C918F5F8C939FBF81E0CA
:107C800090E0DF91CF910895FC0180818823E9F392
:107C9000CF010E94FA3D90E00895FC018081882385
:107CA00019F48FEF9FEF0895CF010E94FA3D90E005
:107CB00008959FB7F8948091C9008F778093C90089
:107CC0008091C9008F7B8093C9008091C9008F7D0E
:107CD0008093C9005A9A52985B9A539A1092CD0099
:107CE0008AE28093CC008091C80082608093C800B3
:107CF00088E18093C9008091CA008F778093CA0081
:107D00008091CA008F7B8093CA008091CA008F7DCA
:107D10008093CA008091CA008F7E8093CA008091B0
:107D2000CA00877F8093CA008091C9008B7F8093AF
:107D3000C9008091CA0084608093CA008091CA0003
:107D400082608093CA0002C08091CE008091C800FA
:107D500087FDFACF8091C90080688093C900809127
:107D6000C90080648093C9009FBF08951F920F923D
:107D70000FB60F9211242F933F934F935F936F93FE
:107D80007F938F939F93AF93BF93EF93FF939091C4
:107D9000CE00809100018B3019F4892F0E94EB45B1
:107DA000FF91EF91BF91AF919F918F917F916F91D3
:107DB0005F914F913F912F910F900FBE0F901F90A9
:107DC00018953C98449A1092B2031092980981E059
:107DD0008093990908956091D1057091D205349BE3
:107DE00018C0CB0101969093D2058093D10581599B
:107DF000914008F44DC08091B203882319F081505E
:107E00008093B2038FEF9FEF90936F0380936E0385
:107E10003BC0CB01019789569140B0F56A3071059E
:107E200028F410926F0310926E0315C06A507040D0
:107E300080E090E029E134E040E050E00E949F4A79
:107E40002AE096958795779567952A95D1F770934F
:107E50006F0360936E0380916E0390916F03209186
:107E6000700330917103845E9D4F821B930B68E613
:107E700071E00E94DE4A845B9040909351058093AC
:107E800050058CE08093B2031092D2051092D10578
:107E90008091B2038823E1F48091CF059091D005C1
:107EA0000E94570D8823A1F08091D3049091D404AF
:107EB000892B31F484E690E09093D4048093D3042A
:107EC00084E690E00E944E0D9093D0058093CF05FC
:107ED000089597FD02C041E004C0909581959F4FA1
:107EE0004FEF68E671E00E94DE4AFC018B35910598
:107EF00054F08B5590408A35910538F484EB90E02E
:107F00008E1B9F0BFC0181E00FC0CF01855B904071
:107F10008A35910518F4E45BF04005C088E691E0ED
:107F20008E1B9F0BFC018FEFEE0FFF1FE159FA4FE5
:107F300025913491992787FD9095B901689F90010B
:107F4000699F300D789F300D1124842F992787FD6C
:107F50009095AC01249FC001259F900D349F900DFA
:107F6000112408952AE530E0281B390BC9010E942D
:107F7000693F08951F93CF93DF93EB01672B29F49B
:107F8000009719F480E090E091C097FF02C01FEFC6
:107F900001C011E0209729F48AE51802C0011124DC
:107FA00085C09C01B901882777FD8095982F26E030
:107FB000660F771F881F991F2A95D1F79E014427C6
:107FC00037FD4095542F0E94134BF90137FF03C032
:107FD000F095E195FF4F31E0EA35F30734F4EB5DBE
:107FE000F94F8491282F30E047C04CE1E73AF4077D
:107FF0001CF02AE530E040C059E0ED38F5071CF0F0
:1080000029E530E039C085E0EA3BF8071CF028E5B7
:1080100030E032C024E0E731F2071CF027E530E021
:108020002BC033E0EE32F3071CF026E530E024C02D
:1080300042E0E939F4071CF025E530E01DC052E0CC
:10804000E233F5071CF024E530E016C081E0E73E9E
:10805000F8071CF023E530E00FC021E0ED3AF2070D
:108060001CF022E530E008C0EF57F1401CF021E59C
:1080700030E002C020E530E01C161D066CF4812FB4
:10808000992787FD9095AC01249FC001259F900DF5
:10809000349F900D11240AC011162CF484EB90E04B
:1080A000821B930B03C0C901845B9040DF91CF9189
:1080B0001F9108959F92AF92BF92CF92DF92EF925D
:1080C000FF920F931F935B016C0161157105810590
:1080D000910511F17B018C019924C601B501A8011C
:1080E00097010E94F14A2E0D3F1D401F511F5695CA
:1080F000479537952795E21AF30A040B150B82E092
:10810000E816F1040105110558F0939488E29816D9
:1081100039F079018A01E1CF20E030E040E050E021
:10812000CA01B9011F910F91FF90EF90DF90CF909E
:10813000BF90AF909F900895E091AE08F0E0EE0FF1
:10814000FF1FEA5BF74F0190F081E02DF7FF03C0BE
:10815000F095E195FF4F3F971CF081E090E0089586
:10816000E091AF08F0E0EE0FFF1FEA5BF74F808170
:10817000918120E030E097FF03C0909581959F4F5B
:108180000F9714F021E030E0C90108958091730643
:1081900081508230F0F5809175068330D1F5809161
:1081A000760690917706A0917806B0917906809333
:1081B000E3059093E405A093E505B093E60580916F
:1081C0007A0690917B06A0917C06B0917D06809303
:1081D000E7059093E805A093E905B093EA0580913F
:1081E0007E0690917F06A0918006B09181068093D3
:1081F000EB059093EC05A093ED05B093EE0581E0BF
:108200008093EF0588EE93E09093D4048093D30499
:1082100008951092EF050895809173068150823081
:10822000C0F5809175068330A1F580917606909116
:108230007706A0917806B09179068093D605909341
:10824000D705A093D805B093D90580917A0690916F
:108250007B06A0917C06B0917D068093DA05909311
:10826000DB05A093DC05B093DD0580917E0690913F
:108270007F06A0918006B09181068093DE059093E1
:10828000DF05A093E005B093E10581E08093E2056E
:1082900008951092E20508951092EF050895109246
:1082A0007705109276051092790510927805089559
:1082B0002F923F924F925F926F927F928F929F92F6
:1082C000AF92BF92CF92DF92EF92FF920F931F93E4
:1082D000CF93DF93CDB7DEB760970FB6F894DEBFCC
:1082E0000FBECDBF8C0180917306813009F091C221
:1082F00080917506833009F08CC280916E03909155
:108300006F0397FD86C20115110509F47AC0F801C3
:108310008485882309F475C0823039F48091F20590
:108320009091F3050817190791F11092F805109232
:10833000F9051092FA051092FB051092F4051092BF
:10834000F5051092F6051092F705F8016481758124
:108350008681978120E836E948E950E00E94134B76
:10836000DA01C9010E94B23FAA2797FDA095BA2F52
:108370008093B3039093B403A093B503B093B60373
:108380001093F3050093F20582E0F80184872091B1
:108390007A0630917B0640917C0650917D06F8016B
:1083A00084819581A681B781281B390B4A0B5B0B11
:1083B00029873A874B875C876091760670917706AC
:1083C0008091780690917906208131814281538194
:1083D000621B730B840B950B2091B3033091B40394
:1083E0004091B5035091B6030E949F4A20E030E2CD
:1083F00040E050E00E94134B2D833E834F8358870B
:1084000018C01092F8051092F9051092FA05109212
:10841000FB051092F4051092F5051092F6051092E6
:10842000F70519861A861B861C861D821E821F82EE
:108430001886E090D305FF2400E010E0A090D4055A
:10844000BB24CC24DD2469857A858B859C85A80195
:1084500097010E949F4A20E038E040E050E00E94EF
:10846000134B39014A012091F8053091F9054091EB
:10847000FA055091FB05C601B5010E949F4A20E014
:1084800030E240E050E00E94134B222433242101CB
:10849000221A330A440A550A261837084808590888
:1084A0006D817E818F819885A80197010E949F4AE6
:1084B00020E038E040E050E00E94134B79018A014F
:1084C0002091F4053091F5054091F6055091F7059E
:1084D000C601B5010E949F4A20E030E240E050E032
:1084E0000E94134BAA24BB246501A21AB30AC40A32
:1084F000D50AAE18BF08C00AD10AC601B501A60147
:1085000095010E949F4A7B018C01C201B101A20129
:1085100091010E949F4AE60EF71E081F191FC8010D
:10852000B7010E945A407B018C016A3171058105B7
:108530009105ECF0C201B10129E130E040E050E0EA
:108540000E949F4AA80197010E94134B19012A011A
:10855000C601B50129E130E040E050E00E949F4AA9
:10856000A80197010E94134B59016A0178C06985DF
:108570007A858B859C8520E130E040E050E00E94C8
:10858000134B8091F8059091F905A091FA05B091EF
:10859000FB05280F391F4A1F5B1F2093F8053093F6
:1085A000F9054093FA055093FB0521308DE7380714
:1085B00080E0480780E058072CF080E09DE7A0E0CD
:1085C000B0E009C0205033484F4F5F4F64F480E063
:1085D00093E8AFEFBFEF8093F8059093F905A09370
:1085E000FA05B093FB056D817E818F81988520E12E
:1085F00030E040E050E00E94134B8091F4059091F0
:10860000F505A091F605B091F705280F391F4A1F0F
:108610005B1F2093F4053093F5054093F6055093C6
:10862000F7052130ADE73A07A0E04A07A0E05A0776
:108630002CF080E09DE7A0E0B0E009C02050334876
:108640004F4F5F4F64F480E093E8AFEFBFEF80934C
:10865000F4059093F505A093F605B093F705E09027
:10866000D505FF2400E010E02091860630918706B2
:108670004091880650918906C801B7010E949F4A1F
:1086800020E032E040E050E00E94134B221A330A0F
:10869000440A550A29823A824B825C8220918A06DA
:1086A00030918B0640918C0650918D06C801B70120
:1086B0000E949F4A20E032E040E050E00E94134BCD
:1086C00015012601221A330A440A550A80916E03C5
:1086D00090916F030E94B23F5C01CC24B7FCC09420
:1086E000DC2C80916E0390916F030E94693F3C01E6
:1086F000882477FC8094982CC601B501A2019101D1
:108700000E949F4A7B018C01C401B30129813A81F7
:108710004B815C810E949F4AE61AF70A080B190BED
:10872000C801B70120E030E240E050E00E94134B66
:108730002D873E874F87588BC601B50129813A8125
:108740004B815C810E949F4A7B018C01C401B30173
:10875000A20191010E949F4AE60EF71E081F191FF1
:10876000C801B70120E030E240E050E00E94134B26
:10877000AA24BB246501A21AB30AC40AD50AC601F9
:10878000B501A60195010E949F4A7B018C016D8570
:108790007E858F8598899B01AC010E949F4AE60ED9
:1087A000F71E081F191FC801B7010E945A407B011C
:1087B0008C016E3271058105910504F16D857E8510
:1087C0008F8598892DE230E040E050E00E949F4A7A
:1087D000A80197010E94134B2D873E874F87588B26
:1087E000C601B5012DE230E040E050E00E949F4A12
:1087F000A80197010E94134B59016A012D853E85FE
:108800003093790520937805B0927705A09276058C
:1088100018C0109277051092760510927905109283
:1088200078051092F8051092F9051092FA05109249
:10883000FB051092F4051092F5051092F6051092C2
:10884000F70560960FB6F894DEBF0FBECDBFDF917F
:10885000CF911F910F91FF90EF90DF90CF90BF903D
:10886000AF909F908F907F906F905F904F903F90D0
:108870002F900895863418F41092F10507C0803ABD
:1088800010F481E001C082E08093F10580917306CD
:10889000813079F1813020F0823009F0A7C014C016
:1088A000109277051092760510927905109278054E
:1088B0008091F105882309F499C084E690E09093B3
:1088C000D4048093D304089580919E06882331F0C8
:1088D00080919E06815080939E06089510927705A0
:1088E0001092760510927905109278051092730611
:1088F0000895809175069091F105833009F055C077
:10890000913039F0913008F445C0923009F044C0FC
:1089100021C08091E2058823E9F10E949C408823D0
:1089200069F00E940C411092770510927605109222
:108930007905109278051092F00555C08091F005E8
:10894000873018F58F5F8093F0050E940C4180E01E
:1089500090E01DC08091EF05882349F00E940C41F2
:108960000E949C408823C1F483EE95E010C082E30E
:1089700090E09093D4048093D3048091E2058823FF
:1089800049F00E949C40882339F486ED95E00E94CE
:10899000584129C00E940C4110927705109276052B
:1089A00010927905109278051EC0109277051092EA
:1089B000760510927905109278059923A1F080919F
:1089C000740628EC829FC001112420E436E0281BA5
:1089D000390B37FF02C020E030E02E5C3F4F309370
:1089E000D4042093D30482E0809373060895EF9219
:1089F000FF920F931F9380913006813059F580913B
:108A000006068093750680912B06809374068091EC
:108A1000140690911506A0911606B0911706809342
:108A2000820690938306A0938406B0938506809176
:108A3000240690912506A0912606B09127068093E2
:108A4000960690939706A0939806B093990682E0B5
:108A50008093300680914D06813009F059C02091F5
:108A600031063091320640913306509134068091A0
:108A7000AA069091AB06A091AC06B091AD06790123
:108A80008A01E81AF90A0A0B1B0BE0929A06F09287
:108A90009B0600939C0610939D062093AA06309394
:108AA000AB064093AC065093AD068091350690918D
:108AB0003606A0913706B0913806809376069093DB
:108AC0007706A0937806B093790680913906909145
:108AD0003A06A0913B06B0913C0680937A069093AB
:108AE0007B06A0937C06B0937D0680913D06909115
:108AF0003E06A0913F06B091400680937E0690937B
:108B00007F06A0938006B093810682E080934D0695
:108B100080917206813009F04AC08091560690918A
:108B20005706A0915806B091590680938A069093F3
:108B30008B06A0938C06B0938D068091520690917F
:108B40005306A0915406B0915506809386069093E3
:108B50008706A0938806B093890680915A06909163
:108B60005B06A0915C06B0915D06B095A0959095CE
:108B700081959F4FAF4FBF4F80938E0690938F0686
:108B8000A0939006B093910680916206909163063F
:108B9000A0916406B0916506809392069093930627
:108BA000A0939406B093950682E08093720680911C
:108BB0003006882359F080914D06882339F0809142
:108BC0007206882319F081E0809373061F910F913C
:108BD000FF90EF900895482F8091A906843009F402
:108BE00061C0853050F48130D1F0813098F082300E
:108BF000D9F0833009F0D8C01CC0863009F489C090
:108C0000863008F461C0873009F4AAC0883009F0C2
:108C1000CBC0B3C0453B09F0C4C081E0A6C042361A
:108C200009F0BFC082E0A1C0413009F0BAC083E0C2
:108C30009CC0463061F04231D9F0423009F581E301
:108C400096E09093A4068093A3064D9607C08CEF00
:108C500095E09093A4068093A306C5969093A206F0
:108C60008093A10601979093A00680939F060AC067
:108C70008EE496E09093A4068093A3068596EECFAB
:108C80001092A9068091A906882309F48FC084E078
:108C90008093A906842F8F5F8093A8068F5F8093AF
:108CA000A7060895842F90E09093A6068093A506CA
:108CB0009091A806940F9093A8068091A706890F1B
:108CC0008093A70685E051C0242F30E0322F222761
:108CD0008091A5069091A606820F931F9093A606F9
:108CE0008093A5069091A806940F9093A806809172
:108CF000A706890F8093A706E0919F06F091A00632
:108D00008081813019F40E94F7444BC0108286E0C4
:108D10002CC0E091A306F091A4068091A106909149
:108D2000A206E817F90728F44193F093A406E0930C
:108D3000A3069091A806940F9093A8068091A70689
:108D4000890F8093A7068091A5069091A6060197AA
:108D50009093A6068093A506892B41F587E005C070
:108D60008091A806481721F488E08093A906089509
:108D7000E0919F06F091A00613C08091A706E091B4
:108D80009F06F091A006481759F481E0808395B1C1
:108D9000982795B90E94F7448FEF80939E0601C0F3
:108DA00010821092A90608951092A9060895A8E0CD
:108DB000B0E0EDEDF6E40C94384B7B018C016115CD
:108DC00071058105910519F482E089835AC083E019
:108DD00089838EE1C82ED12CDC82CB82ED82FE828B
:108DE0000F831887C801B7010E944A47BC01615030
:108DF000704077FF33C0EE27FF27E61BF70B20E01C
:108E000030E040E050E081E090E0A0E0B0E00E2EE5
:108E100004C0880F991FAA1FBB1F0A94D2F701979D
:108E2000A109B1098E219F21A023B1230097A1059B
:108E3000B10521F021E030E040E050E004C016959B
:108E40000795F794E794EA95D2F72E293F29402B0E
:108E5000512B2D833E834F8358870FC061157105B9
:108E600081F0062E04C0EE0CFF1C001F111F0A9497
:108E7000D2F7ED82FE820F831887C61AD70ADC82EA
:108E8000CB821A82CE0101960E949747E8E028968D
:108E90000C94544BEF92FF920F931F939B01AC01E4
:108EA000203080E0380781E0480780E0580780F4F0
:108EB0002F3F31054105510509F020F4EE24FF2430
:108EC000870119C068E0E62EF12C012D112D13C089
:108ED000203080E0380780E0480781E0580730F410
:108EE00090E1E92EF12C012D112D05C088E1E82E2D
:108EF000F12C012D112D80E290E0A0E0B0E08E1960
:108F00009F09A00BB10B04C056954795379527953F
:108F1000EA94D2F7F901E954FC4F2081821B9109B0
:108F2000A109B1091F910F91FF90EF9008959F92B1
:108F3000AF92BF92CF92DF92EF92FF920F931F9367
:108F4000EE24FF248701FC0124813581468157816D
:108F500091808081823010F44061A2C0843009F495
:108F60009BC0823029F420E030E040E050E005C0B2
:108F7000211531054105510519F4E0E0F0E092C0FA
:108F8000828193816FEF823896070CF05AC062E8B5
:108F90007FEF681B790B6A3171052CF020E030E01F
:108FA00040E050E02AC0AA24BB24650181E090E0A3
:108FB000A0E0B0E0062E04C0880F991FAA1FBB1FB7
:108FC0000A94D2F70197A109B10982239323A4231C
:108FD000B5230097A105B10529F071E0A72EB12CAA
:108FE000C12CD12C04C056954795379527956A9585
:108FF000D2F72A293B294C295D29DA01C9018F774B
:109000009070A070B07080349105A105B10539F45D
:1090100027FF09C0205C3F4F4F4F5F4F04C0215CCA
:109020003F4F4F4F5F4F80E090E0203060E03607C9
:1090300060E0460760E4560710F081E090E0FC0134
:1090400023C08038910544F5FC01E158FF4FDA0157
:10905000C9018F779070A070B07080349105A10520
:10906000B10539F427FF09C0205C3F4F4F4F5F4FD8
:1090700004C0215C3F4F4F4F5F4F57FF05C05695CF
:10908000479537952795319687E0569547953795BB
:1090900027958A95D1F706C020E030E040E050E007
:1090A000EFEFF0E0E22EF32E942F9F77802F807861
:1090B000892B9E2F9795992797958F77082F092BA6
:1090C0009E2F9695812F8078892B97949924979439
:1090D0008F77182F1929C801B7011F910F91FF90A1
:1090E000EF90DF90CF90BF90AF909F900895FC01DC
:1090F0004150504030F001900616D1F73197CF0122
:1091000008958827992708955058BB27AA270ED07D
:1091100079C16AD130F06FD120F031F49F3F11F462
:109120001EF45FC10EF4E095E7FB55C1E92F7BD13A
:1091300080F3BA17620773078407950718F071F474
:109140009EF593C10EF4E0950B2EBA2FA02D0B01C6
:10915000B90190010C01CA01A0011124FF27591B7C
:1091600099F0593F50F4503E68F11A16F040A22F82
:10917000232F342F4427585FF3CF469537952795F3
:10918000A795F0405395C9F77EF41F16BA0B620BF2
:10919000730B840BBAF09150A1F0FF0FBB1F661F39
:1091A000771F881FC2F70EC0BA0F621F731F841F7C
:1091B00048F4879577956795B795F7959E3F08F0A2
:1091C000B3CF9395880F08F09927EE0F9795879561
:1091D00008950CD017C10FD140F006D130F021F422
:1091E0005F3F19F0F8C0511141C1FBC01CD198F389
:1091F0009923C9F35523B1F3951B550BBB27AA2718
:1092000062177307840738F09F5F5F4F220F331F89
:10921000441FAA1FA9F333D00E2E3AF0E0E830D055
:1092200091505040E695001CCAF729D0FE2F27D058
:10923000660F771F881FBB1F261737074807AB0726
:10924000B0E809F0BB0B802DBF01FF2793585F4F9B
:109250002AF09E3F510568F0BEC008C15F3FECF3A5
:10926000983EDCF3869577956795B795F7959F5F60
:10927000C9F7880F911D9695879597F90895E1E0B4
:10928000660F771F881FBB1F621773078407BA0713
:1092900020F0621B730B840BBA0BEE1F88F7E0956E
:1092A000089504D06894B111E1C00895C4D088F045
:1092B0009F5790F0B92F9927B751A0F0D1F0660FC2
:1092C000771F881F991F1AF0BA95C9F712C0B130DD
:1092D00081F0CBD0B1E00895C8C0672F782F8827E0
:1092E000B85F39F0B93FCCF3869577956795B3951C
:1092F000D9F73EF490958095709561957F4F8F4F8B
:109300009F4F0895E89409C097FB3EF4909580958F
:10931000709561957F4F8F4F9F4F9923A9F0F92F3B
:1093200096E9BB279395F695879577956795B795B9
:10933000F111F8CFFAF4BB0F11F460FF1BC06F5F9F
:109340007F4F8F4F9F4F16C0882311F096E911C0B1
:10935000772321F09EE8872F762F05C0662371F0D2
:1093600096E8862F70E060E02AF09A95660F771FE6
:10937000881FDAF7880F9695879597F9089507D093
:1093800008F481E0089503D008F48FEF0895990F51
:109390000008550FAA0BE0E8FEEF16161706E807BF
:1093A000F907C0F012161306E407F50798F0621BE0
:1093B000730B840B950B39F40A2661F0232B242BB5
:1093C000252B21F408950A2609F4A140A6958FEFD4
:1093D000811D811D089597F99F6780E870E060E026
:1093E00008959FEF80EC089500240A94161617063E
:1093F00018060906089500240A9412161306140686
:1094000005060895092E0394000C11F4882352F0E8
:10941000BB0F40F4BF2B11F460FF04C06F5F7F4FA0
:109420008F4F9F4F089557FD9058440F551F59F087
:109430005F3F71F04795880F97FB991F61F09F3F41
:1094400079F087950895121613061406551FF2CF6A
:109450004695F1DF08C0161617061806991FF1CFBA
:1094600086957105610508940895E894BB276627E1
:109470007727CB0197F908950BD0C4CFB5DF28F03B
:10948000BADF18F0952309F0A6CFABCF1124EECFA9
:10949000CADFA0F3959FD1F3950F50E0551F629F4F
:1094A000F001729FBB27F00DB11D639FAA27F00D3D
:1094B000B11DAA1F649F6627B00DA11D661F829F64
:1094C0002227B00DA11D621F739FB00DA11D621F49
:1094D000839FA00D611D221F749F3327A00D611D66
:1094E000231F849F600D211D822F762F6A2F112448
:1094F0009F5750408AF0E1F088234AF0EE0FFF1F9B
:10950000BB1F661F771F881F91505040A9F79E3FD1
:10951000510570F060CFAACF5F3FECF3983EDCF3CB
:10952000869577956795B795F795E7959F5FC1F70E
:10953000FE2B880F911D9695879597F90895629F48
:10954000D001739FF001829FE00DF11D649FE00D3B
:10955000F11D929FF00D839FF00D749FF00D659F9C
:10956000F00D9927729FB00DE11DF91F639FB00D9B
:10957000E11DF91FBD01CF0111240895991B79E068
:1095800004C0991F961708F0961B881F7A95C9F793
:1095900080950895AA1BBB1B51E107C0AA1FBB1FE2
:1095A000A617B70710F0A61BB70B881F991F5A956F
:1095B000A9F780959095BC01CD01089597FB092EE0
:1095C00007260AD077FD04D0E5DF06D000201AF484
:1095D000709561957F4F0895F6F7909581959F4F0F
:1095E0000895A1E21A2EAA1BBB1BFD010DC0AA1FE4
:1095F000BB1FEE1FFF1FA217B307E407F50720F0FC
:10960000A21BB30BE40BF50B661F771F881F991F76
:109610001A9469F760957095809590959B01AC01BF
:10962000BD01CF01089597FB092E05260ED057FDE9
:1096300004D0D7DF0AD0001C38F4509540953095FF
:1096400021953F4F4F4F5F4F0895F6F790958095C6
:10965000709561957F4F8F4F9F4F08952F923F9246
:109660004F925F926F927F928F929F92AF92BF9232
:10967000CF92DF92EF92FF920F931F93CF93DF93DE
:10968000CDB7DEB7CA1BDB0B0FB6F894DEBF0FBE3B
:10969000CDBF09942A88398848885F846E847D8488
:1096A0008C849B84AA84B984C884DF80EE80FD808A
:1096B0000C811B81AA81B981CE0FD11D0FB6F89400
:1096C000DEBF0FBECDBFED010895F999FECFB2BD4B
:1096D000A1BDF89A119600B40895F7DF01921A948B
:1096E000E1F70895F2DFE02DF0DFF02D0895F9990C
:1096F000FECFB2BDA1BD00BC11960FB6F894FA9A88
:10970000F99A0FBE0895F3DF012CF1DF11240895BB
:0C9710000190EDDF1A94E1F70895FFCFFF
:10971C000AFF0164496E74656772616C4E69636B14
:10972C0020202020496E74656772616C526F6C6CDE
:10973C00202020204163634E69636B202020202071
:10974C0020202020416363526F6C6C20202020204D
:10975C00202020204779726F59617720202020200B
:10976C002020202052656164696E674865696768CE
:10977C00742020204163635A2020202020202020A8
:10978C002020202047617320202020202020202012
:10979C00202020205265636569766572204C6576C1
:1097AC00656C2020566F6C7461676520202020202A
:1097BC00202020204D6F746F722046726F6E744C97
:1097CC00656674204D6F746F722046726F6E7452A2
:1097DC00696768744D6F746F7220526561724C6565
:1097EC00667420204D6F746F7220526561725269DD
:1097FC00676874204D6F746F7220526967687420AB
:10980C00202020204D6F746F72204C6566742020D0
:10981C00202020204163635F5A202020202020201C
:10982C0020202020535049204572726F7220202036
:10983C0020202020535049204F6B20202020202016
:10984C00202020202020202020202020202020200C
:10985C0020202020536572766F202020202020208D
:10986C00202020204E69636B2020202020202020E7
:10987C0020202020526F6C6C2020202020202020C3
:10988C0020202020202020202020202020202020CC
:10989C0020202020202020202020202020202020BC
:1098AC0020202020202020202020202020202020AC
:1098BC00202020202020202020202020202020209C
:1098CC00202020202020202020202020202020208C
:1098DC00202020202020202020202020202020207C
:1098EC00202020202020202020202020202020206C
:1098FC00202020204750535F4E69636B202020208E
:10990C00202020204750535F526F6C6C2020202069
:10991C0020202020FFFF010A6400007D0000FF03CF
:10992C000102030405060708090A48656C6C6F20E0
:10993C00576F726C64000000000000000000000013
:10994C00000000000000000000000000000000000B
:10995C0000000000000000000000000000000000FB
:10996C0000000000000000000000000000000000EB
:10997C00000000000000000000000C016400FFFF6C
:10998C00FFFFF40190D0030090D00300ECFF17B759
:10999C00D13830FB103A409696020A0000000000C5
:1099AC00000000644600006401426567696E6E65E4
:1099BC007200004E6F726D616C000053706F7274A8
:1099CC0000000C0100000000010202030303030469
:1099DC000404040404040405050505050505050532
:1099EC000505050505050506060606060606060612
:1099FC0006060606060606060606060606060606FB
:109A0C0006060606060606070707070707070707E1
:109A1C0007070707070707070707070707070707CA
:109A2C0007070707070707070707070707070707BA
:109A3C0007070707070707070707070707070707AA
:109A4C000707070707070708080808080808080891
:109A5C00080808080808080808080808080808087A
:109A6C00080808080808080808080808080808086A
:109A7C00080808080808080808080808080808085A
:109A8C00080808080808080808080808080808084A
:109A9C00080808080808080808080808080808083A
:109AAC00080808080808080808080808080808082A
:109ABC00080808080808080808080808080808081A
:089ACC0008080808080808005A
:00000001FF
